:100000004AEF3FF09280000C046ED8CF05F0E0CFAD
:1000100006F00001E9CF0CF0EACF07F0E1CF08F0DD
:10002000E2CF09F0D9CF0AF0DACF0BF0F3CF12F01C
:10003000F4CF13F0FACF14F0F5CF15F0F6CF16F099
:10004000F7CF17F000C00EF001C00FF002C010F0A3
:1000500003C011F0F2AA30EF00F0F2B48AEF1DF005
:100060000EC000F00FC001F010C002F011C003F08C
:100070000CC0E9FF07C0EAFF078E08C0E1FF09C016
:10008000E2FF0AC0D9FF0BC0DAFF12C0F3FF13C0B2
:10009000F4FF14C0FAFF15C0F5FF16C0F6FF17C035
:1000A000F7FF045006C0E0FF05C0D8FF1000F76A54
:1000B000BE0FF66E000EF7220900F5501200191A55
:1000C0001B1C1D2425263038393F406B6C6D7A7C13
:1000D0007D7E7F00E20FF66E000EF7220900F550DC
:1000E000120007DBCD79604DD5003070391662AF54
:1000F000FDDDCA5ECA040007DBCD79604DD5303026
:10010000703916625AF98B5D5E5D040007DBCD79AC
:10011000604DD5503070391662F76D3BB45EB40453
:100120000007DBCD79604E76103070391662364E9E
:100130005FD25ED2040007DBCD796053BC90307093
:1001400039166244F9E7F85EF8040007DBCD796000
:1001500053BCB03070391662DEB793785E78040015
:1001600007DBCD796053BED03070391662367AC85D
:10017000645E64040007DBCD796053C5B03070392C
:100180001662E15C06405E40040007DBCD796053F7
:10019000C8D03070391662DCE0EE445E44040007DB
:1001A000DBCD796053CAE03070391662D12A80DF26
:1001B0005EDF040007DBCD796053D1403070391623
:1001C000622200E6DB5EDB040007DBCD796053D101
:1001D000503070391662F376179D5E9D040007DB80
:1001E000CD796053D1A0307039166268CB15495E65
:1001F00049040007DBCD796053DC5030703916625A
:10020000A16ED11C5E1C040007DBCD796053DC704D
:100210003070391662409281715E71040007DBCD47
:10022000796053E1E03070391662CEB60DFA5EFAAD
:10023000040007DBCD796053E5003070391662EEBB
:1002400070A7525E52040007DBCD796053E880301E
:10025000703916622B209B765E76040007DBCD7921
:100260006053E8A03070391662FE3AEFED5EED049F
:100270000007DBCD796053E8F030703916623059F1
:100280008C735E73040007DBCD796053ED603070D2
:1002900039166271AEA5795E79040007DBCD79600D
:1002A00053EDD03070391662B86835565E5604008A
:1002B00007DBCD7960540040307039166256AEC409
:1002C000F55EF5040007DBCD7960540230307039FB
:1002D000166227614AB75EB7040007DBCD79605428
:1002E00002703070391662BC6B517D5E7D04000770
:1002F000DBCD79605405A03070391662BC6952AB11
:100300005EAB040007DBCD79605409B0307039165C
:10031000623CBACF795E79040007DBCD7960540D79
:1003200000307039166239D9BDD95ED9040007DBB7
:10033000CD79605413503070391662F42208145E7F
:1003400014040007DBCD79605429403070391662FF
:10035000DC418EF35EF3040007DBCD796054296045
:1003600030703916628A8F1DD85ED8040007DBCD45
:100370007960542F30307039166261D6E4C55EC59D
:10038000040007DBCD79605431A03070391662F17A
:1003900057C27C5E7C040007DBCD7960543AE030C4
:1003A00070391662CA318C245E24040007DBCD79D3
:1003B00060543B0030703916628AA4C15D5E5D04F2
:1003C0000007DBCD7960543B1030703916622D4345
:1003D0005C905E90040007DBCD79605444903070EF
:1003E0003916625C4287C45EC4040007DBCD7960C5
:1003F0005446703070391662FBF150E55EE504003A
:1004000007DBCD79605449D030703916628BA13347
:10041000095E09040007DBCD79605449E03070398A
:100420001662D71146A05EA0040007DBCD796054A8
:1004300049F03070391662F50D935B5E5B0400077E
:10044000DBCD7960544A003070391662C6DD3EE675
:100450005EE6040007DBCD796054558030703916B4
:10046000628CE100315E31040007DBCD79605458C5
:10047000E03070391662F0BA067D5E7D040007DB5D
:10048000CD7960545A9030703916629252A6255E2A
:1004900025040007DBCD79605460B03070391662F6
:1004A000333A71215E21040007DBCD79605462404C
:1004B00030703916623A05CB5F5E5F040007DBCD12
:1004C000796054625030703916627CFF50685E6803
:1004D000040007DBED7D606619E03070391662A517
:1004E0001F9D4D5E4D080007DBED7D60661A5030A4
:1004F00070391662D6F2EB1A5E1A04001152EC4DF6
:10050000802E1EC43B51B9166208C588AC5EAC048F
:10051000001152EC4D802F0E244151B51662F79E0A
:1005200057505E5004001152EC4D802F33142C5163
:10053000B516623263F1AE5EAE040021528B4D609F
:10054000459AF02C465D166284D4B9885E88040012
:1005500021528B4D604B95443E469D1662E965D312
:10056000595E59040000740FF66E050EF72209005B
:10057000F550120007DBCD796046C5D03170051704
:1005800046D4B687485E48040007DBCD796046C98B
:10059000C0317005174631765BAD5EAD040007DBF8
:1005A000CD796046C9F031700517460FA820065E68
:1005B00006040007DBCD796046D1D03170051746BF
:1005C000E19233F95EF9040007DBCD796046D4E0AF
:1005D000317005174681B03B865E86040007DBCD8F
:1005E000796046D50031700517464EF4FB2C5E2C21
:1005F000040007DBCD796046D5103170051746251C
:10060000891CCD5ECD040007DBCD796046DA303140
:100610007005174639E955D75ED7040007DBCD7959
:100620006046DA4031700517467538E8875E870402
:100630000007DBCD796046DA603170051746011C92
:10064000736C5E6C040007DBCD796046DA90317024
:10065000051746FF2733115E110C0007DBCD7960CB
:1006600046DDF031700517460CB6FFD05ED00400B1
:1006700007DBCD796046DE20317005174667D970FB
:10068000885E88040007DBCD796046E1F0317005B3
:100690001746CDC347E05EE0040007DBCD79604636
:1006A000E890317005174668484DAD5EAD0400070F
:1006B000DBCD796046E8A031700517469B22F9B082
:1006C0005EB0040007DBCD796046EB103170051792
:1006D00046D4D05A1D5E1D040007DBCD796046EB81
:1006E000503170051746B1078D385E38040007DBBE
:1006F000CD796046EB603170051746C53B8C415E95
:1007000041040007DBCD796046EE90317005174655
:10071000F196D5745E74040007DBCD7960470490D0
:100720003170051746243CC3F65EF6040007DBCDA6
:1007300079604704B03170051746149572FE5EFE6D
:10074000040007DBCD79604704C031700517462AE5
:1007500063291D5E1D040007DBCD79604708503119
:100760007005174675BE163C5E3C040007DBCD796C
:10077000604708803170051746F74C71FB5EFB043B
:100780000007DBCD79604708B03170051746DFB14F
:1007900078175E17040007DBCD79604708C0317019
:1007A00005174623F8A70D5E0D040007DBCD796021
:1007B000470EE031700517461BEB47E05EE0040092
:1007C00007DBCD79604711E03170051746B1CAFCEF
:1007D000CF5ECF040007DBCD796047120031700592
:1007E000174676C184985E98040007DBCD79604790
:1007F00015C03170051746CF0B923A5E3A040007D8
:10080000DBCD79604718A03170051746A3C689ED86
:100810005EED040007DBCD7960471DE03170051700
:10082000468680F9BB5EBB0400081BCD7960471E7D
:100830000031700517469598CFA85EA8040007DB25
:10084000CD7960471E40317005174686DCEE535E59
:1008500053040007DBCD79604721B031700517469E
:100860009D54C8295E29040007DBCD7960472650D6
:1008700031700517464371639E5E9E040007DBCD11
:1008800079604726803170051746F1DB91A45EA49C
:10089000040007DBCD79604726903170051746CA02
:1008A0006CC8615E61040007DBCD79604729703157
:1008B000700517464696EBDB5EDB040007DBCD795F
:1008C000604729A03170051746CD73B23C5E3C04E9
:1008D0000007DBCD7960472C2031700517469B1F40
:1008E00097A65EA6040007DBCD7960472E403170E5
:1008F0000517465E2B01A35EA3040007DBCD7960DC
:10090000472E5031700517467F51DF365E360400A2
:1009100007DBCD7960472E9031700517463CD3C771
:100920002F5E2F040007DBCD79604731B0317005B1
:10093000174672D054CE5ECE040007DBCD796047F7
:1009400031D03170051746A729499F5E9F040007E3
:10095000DBCD79604736D0317005174642086570A7
:100960005E70040007DBCD79604736E03170051713
:100970004636F1D77F5E7F040007DBCD7960473EC6
:10098000A0317005174642F492035E030400215122
:100990006B216043C5C443269D174656F258AE5E90
:1009A000AE040011530C45808B5110355181174610
:1009B00067FCC9445E44040011530C49808F410414
:1009C0002E518D1746F116C9235E23040000DC0F5B
:1009D000F66E090EF7220900F550120007E3ED7DCF
:1009E00060688950316005165699763AF65EF604CD
:1009F0000007E3ED7D606889803160051656B2011D
:100A0000FCBC5EBC040007E3ED7D6068899031604A
:100A10000516564EACE0085E08040007E3ED7D6065
:100A20006889A031600516566F5D44A55EA5040077
:100A300007E3ED7D6068911031600516561E705217
:100A4000475E47040007E3ED7D6068915031600523
:100A500016568ED9FF935E93040007E3ED7D606820
:100A600091603160051656401AA6F75EF70400073C
:100A7000E3ED7D6068931031600516561BEB9C1505
:100A80005E15040007E3ED7D606893203160051674
:100A900056C7EB3F5A5E5A040007E3ED7D60689647
:100AA00040316005165640104C305E30040007E3BC
:100AB000ED7D60689D1031600516562B64655D5EA6
:100AC0005D040007E3ED7D60689EC0316005165649
:100AD00002E623635E63040007E3ED7D60689F1018
:100AE0003160051656EB89A5B25EB2040007E3ED4E
:100AF0007D6068A2103160051656FFC75E2E5E2E1F
:100B0000040007E3ED7D6068A22031600516568081
:100B1000B5622F5E2F040007E3ED7D6068A25031BF
:100B20006005165602F7D12C5E2C040007E3ED7D1C
:100B30006068A5903160051656180A8A575E5704FA
:100B40000007E3ED7D6068A71031600516567C80D4
:100B500067D65ED6040007E3ED7D6068A7203160AC
:100B60000516561BBBE33E5E3E040007E3ED7D60C9
:100B700068AA003160051656A37B7EF65EF6040077
:100B800007E3ED7D6068AE303160051656FFCFC8D3
:100B90009C5E9C040007E3ED7D6068B190316005C8
:100BA00016569239EF9F5E9F040007E3ED7D606863
:100BB000B4B03160051656144FF85D5E5D04000751
:100BC000E3ED7D6068B4E0316005165631CAE5B0EA
:100BD0005EB0040007E3ED7D6068B4F03160051697
:100BE000568119FFD95ED9040007E3ED7D6068B630
:100BF000C03160051656AE1C06385E38040007E3A7
:100C0000ED7D6068BDE03160051656B4DB15DD5E34
:100C1000DD040007E3ED7D6068BE10316005165607
:100C2000204B7D425E42040007E3ED7D6068C59085
:100C3000316005165604826E475E47040007E3EDF7
:100C40007D6068CED03160051656E617998C5E8CB3
:100C5000040007E3ED7D6068CF303160051656254E
:100C60001B3B005E00040007E3ED7D6068D190311E
:100C7000600516563D2263C75EC7040007E3ED7D9D
:100C80006068D5C03160051656C0D68B725E72049E
:100C90000007E3ED7D6068D5D03160051656C3616D
:100CA000DF825E82040007E3ED7D6068DF30316043
:100CB000051656A9D66C065E06040007E3ED7D60B6
:100CC00068E5A031600516565581167D5E7D0400ED
:100CD00007E3ED7D6068E5B03160051656EB31C67F
:100CE000B35EB3040007E3ED7D6068E5C0316005E5
:100CF0001656217B3FBA5EBA040007E3ED7D6068BB
:100D0000E5D03160051656AB79F7EA5EEA040007D4
:100D1000E3ED7D6068E84031600516560843061F24
:100D20005E1F040007E3ED7D6068E8703160051622
:100D300056689463FD5EFD040007E3ED7D6068EA9C
:100D4000A031600516564B8A7E0F5E0F040007E344
:100D5000ED7D606904F03160051656159BA5245E93
:100D600024040007E3ED7D60690700316005165635
:100D70005CF5A9FC5EFC040007E3ED7D60690730CB
:100D80003160051656C586931C5E1C040007E3ED12
:100D90007D606907503160051656783B01EE5EEEC6
:100DA000040007E3ED7D60690C903160051656255F
:100DB000A7CB2E5E2E040007E3ED7D60690D0031A8
:100DC0006005165661A93E005E00040007E3ED7D54
:100DD00060690EB0316005165601F8BA065E060469
:100DE0000007E3ED7D606919D03160051656BEF14C
:100DF00034495E49040011538C49804D7010415FA5
:100E0000D1165641BDD71C5E1C040011538C49807D
:100E10004D71A4415FD116560978B1425E4204007B
:100E200021524B456096D7903A40051656BBB436D2
:100E3000585E58040000440FF66E0E0EF7220900AB
:100E4000F550120007EB6D6D606726303D9AD516A0
:100E5000520CCFC31D5E1D040007EBCD79604CC65C
:100E6000803D9AD51652026F50EF5EEF040007E303
:100E7000CD79604CC6903D9AD516524E4EB6705EF6
:100E800070080007E3CD79604CD1303D9AD51652F9
:100E90009D8283E15EE1040007E3CD79604CD610CA
:100EA0003D9AD516520A1839715E71040007EBCDD0
:100EB00079604CD6303D9AD516529FEDBDBD5EBDD2
:100EC00004000803CD79604CD9C03D9AD51652D99B
:100ED000035AEA5EEA040007E3CD79604CE1F03D95
:100EE0009AD516520C3A12A95EA9040007E3CD79EF
:100EF000604CE5903D9AD51652B8A795635E6304A1
:100F00000007E3CD79604CE5B03D9AD51652C2D7C3
:100F1000C21E5E1E040007E3CD79604CE8603D9A76
:100F2000D516525950D0CD5ECD040007E3CD79607F
:100F30004CEC503D9AD516526EACE4065E060400A9
:100F400007E3CD79604CEC703D9AD5165256F95FA7
:100F5000F05EF0040007E3CD79604CEC903D9AD54B
:100F6000165258F8FABA5EBA040007E3CD79604C1D
:100F7000EE203D9AD5165247B6DA795E790400071D
:100F8000E3CD79604D01F03D9AD51652C903E54392
:100F90005E43040007E3CD79604D02103D9AD516FB
:100FA0005223F0663A5E3A040007E3CD79604D07BC
:100FB000203D9AD5165246981F7B5E7B040007E3BE
:100FC000CD79604D09E03D9AD516524EF036FC5E63
:100FD000FC040007E3CD79604D0A003D9AD5165216
:100FE00068906A055E05040007E3CD79604D0DB099
:100FF0003D9AD51652DED03D135E13040007E3CDB3
:1010000079604D10703D9AD51652D1BCCC5C5E5CB7
:10101000040007E3CD79604D14803D9AD516523E09
:1010200092CE6B5E6B040007E3CD79604D1DD03D21
:101030009AD5165240289CA45EA4040007E3CD79FB
:10104000604D1DF03D9AD51652DE74558F5E8F04AB
:101050000007E3CD79604D28503D9AD516527D6F3B
:101060007D8A5E8A040007E3CD79604D28A03D9A11
:10107000D51652130405075E07040007E3CD796017
:101080004D2A203D9AD516522890C3EC5EEC040000
:1010900007E3CD79604D34B03D9AD516527DA091CD
:1010A000555E55040007E3CD79604D37203D9AD554
:1010B00016528162CFA65EA6040007E3CD79604D8B
:1010C0003EC03D9AD5165296C17E4A5E4A0400073C
:1010D000E3CD79604D3EE03D9AD51652B3AB49124F
:1010E0005E12040007E3CD79604D3F003D9AD516AE
:1010F00052403932E95EE9040007E3CD79604D459D
:10110000803D9AD5165240EEB84E5E4E040007E37D
:10111000CD79604D73303D9AD516520E6550E55E1F
:10112000E5040007E3CD79604D73403D9AD5165232
:10113000AE0B13185E18040007E3CD79604D7350B1
:101140003D9AD516521D18DC675E67040007E3CD93
:1011500079604D7D403D9AD516523240B5675E6745
:10116000040007E3CD79604D80A03D9AD516526FFB
:10117000CA40585E58040007E3CD79604D80B03D09
:101180009AD51652C84A83AC5EAC040007E3CD7909
:10119000604D80C03D9AD5165245B3D5FE5EFE0423
:1011A0000007E3CD79604D80D03D9AD516520801F5
:1011B00067A35EA3040007E3CD79604D80E03D9A0C
:1011C000D51652F1FEB7455E45040007E3CD7960C0
:1011D0004D84903D9AD5165291F2769C5E9C040007
:1011E00007E3CD79604D88B03D9AD5165247BEDEF3
:1011F000825E82040007E3CD79604D88C03D9AD5B8
:1012000016523212F4015E01040007E3CD79604DFD
:101210008A403D9AD51652B64605A25EA204000742
:10122000E3CD79604D8E503D9AD516526681A20667
:101230005E06040007E3CD79604D8E603D9AD516B9
:1012400052CE955B735E73040007E3CD79604D91D8
:10125000D03D9AD51652915866735E73040007E329
:10126000CD79604D99C03D9AD516521F8B55055EBC
:10127000050400215A4B4560673694353FD5165218
:101280008E217A485E480400115B6C4D80CFBFB060
:101290003E5F91165236EBE4705E700400115B6C99
:1012A0004D80D061443A5F911652B99F9AC65EC68E
:1012B0000400C00FF66E120EF7220900F55012005E
:1012C000081BED7D60668670276FC116664DF5259B
:1012D000C35EC30400081BED7D60668F80276FC16D
:1012E0001666A55BF7AE5EAE0400081BED7D60667A
:1012F0009480276FC11666ED88954C5E4C040008FB
:101300001BED7D60669490276FC11666177B418147
:101310005E810400081BED7D60669700276FC11693
:101320006655B301D85ED80400081BED7D6066C029
:1013300060276FC11666622FE8AD5EAD0400081B22
:10134000ED7D6066C080276FC11666B6E1D26D5E26
:101350006D0400081BED7D6066C2C0276FC1166674
:101360003415A12A5E2A0400081BED7D6066C33097
:10137000276FC11666D5B86B5D5E5D0400081BED76
:101380007D6066C660276FC11666A0D7265F5E5F68
:101390000400081BED7D6066C9A0276FC116669B1F
:1013A000F6FF535E530400081BED7D6066C9E0271D
:1013B0006FC116666C8382EC5EEC0400081BED7D49
:1013C0006066C9F0276FC11666B001AC8C5E8C04F4
:1013D00000081BED7D6066D1C0276FC11666E5531E
:1013E000EAE55EE50400081BED7D6066D630276FF8
:1013F000C116668CD07D6F5E6F0400081BED7D60AA
:1014000066D940276FC116668A8B25155E150400C4
:10141000081BED7D6066D980276FC11666EB9D5075
:10142000D75ED70400081BED7D6066D9B0276FC179
:101430001666750F2D965E960400081BED7D60669E
:10144000DC90276FC1166637A15E2C5E2C04000865
:101450001BED7D6066DCC0276FC11666A1E959A54A
:101460005EA50400081BED7D6066DCD0276FC11609
:101470006633B00C2B5E2B0400081BED7D6066E02C
:1014800060276FC116661B2465725E720400081B1C
:10149000ED7D6066E4B0276FC11666A85841415ED5
:1014A000410800081BED7D6066EAD0276FC1166613
:1014B000E92C5F085E080400081BED7D6066EAF019
:1014C000276FC116669B94AA175E170400081BEDD0
:1014D0007D6066EB00276FC1166607E63B995E9953
:1014E0000400081BED7D6066EDC0276FC116661114
:1014F0003E913B5E3B0400081BED7D606704402786
:101500006FC11666285D22BA5EBA0400081BED7D25
:1015100060670450276FC11666FC618BEB5EEB04BD
:1015200000081BED7D60670480276FC11666D5B289
:1015300088C25EC20400081BED7D606704B0276F9F
:10154000C11666DDD0C8D85ED80400081BED7D60EA
:10155000670730276FC11666713631E85EE8040010
:10156000081BED7D60670750276FC11666AFE0343A
:10157000855E850400081BED7D606711A0276FC1A3
:101580001666C20E29FD5EFD0400081BED7D606736
:101590001530276FC116668582169D5E9D04000872
:1015A0001BED7D60671750276FC11666558AE1D025
:1015B0005ED00400081BED7D60671790276FC11691
:1015C00066C6661D935E930400081BED7D60671C74
:1015D000E0276FC1166680C27D6A5E6A0400081B40
:1015E000ED7D60671D40276FC11666EC0A796B5E62
:1015F0006B0400081BED7D60672110276FC1166624
:1016000086A3318C5E8C0400081BED7D6067212071
:10161000276FC11666446452DA5EDA0400081BEDD7
:101620007D606724C0276FC11666BCFABEB55EB583
:101630000400081BED7D606726C0276FC116662574
:10164000EA6EEE5EEE0400081BED7D606726F02773
:101650006FC11666B43CAC5B5E5B0400081BED7D9D
:1016600060672A30276FC11666943AF1EC5EEC048D
:1016700000081BED7D60673440276FC11666765EFB
:10168000C83D5E3D0400081BED7D606734B0276FE8
:10169000C11666F1FBD1F65EF60400081BED7D6015
:1016A000673690276FC11666A8E58ECC5ECC040025
:1016B000081BED7D60673700276FC116667AF93425
:1016C000295E290400081BED7D606741C0276FC1BA
:1016D0001666D36D87115E110400115B6C49802C76
:1016E00019602F600916663EFF1B825E820400119E
:1016F0005B6C55802C52042C60091666C495132A25
:101700005E2A0400215A6B49607664E03B43A916C7
:1017100066A3EAA5525E52040000280FF66E170E6B
:10172000F7220900F5501200081BED7D60698A2040
:10173000319D591742EE35F0425E420800081BED1C
:101740007D60698A30319D5917421D8F5ABD5EBD3B
:101750000400081BED7D60698EA0319D5917427011
:10176000E1D6A65EA60400081BED7D60698EC0313F
:101770009D591742525898135E130400081BED7DC3
:10178000606991D0319D591742BC7E34785E7804EF
:10179000001BC24B4560673694353FD51652F78D16
:1017A00089C200C20000081BED7D60699220319D56
:1017B000591742FA5D6BB15EB10400081BED7D6004
:1017C000699230319D5917423411EFA75EA704008A
:1017D000081BED7D60699520319D5917425D27FEFC
:1017E000FE5EFE0400081BED7D60699540319D5949
:1017F0001742C7E94D795E790400081BED7D6069E9
:101800009C70319D591742BAE0D3AA5EAA04000821
:101810001BED7D60699CC0319D591742A5495F2031
:101820005E200400081BED7D60699EE0319D591724
:1018300042ED2F5D2E5E2E0400081BED7D60699E3B
:10184000F0319D591742F551BCB95EB90400081B2F
:10185000ED7D6069A1C0319D591742AA32A99F5EF2
:101860009F0400081BED7D6069A520319D5917423A
:1018700055C00ED15ED10400081BED7D6069AB1030
:10188000319D591742A4A661175E170400081BED8D
:101890007D6069AB40319D591742B30D41DB5EDB82
:1018A0000400081BED7D6069AB60319D59174257FC
:1018B000A15FAD5EAD0400081BED7D6069AE103127
:1018C0009D591742641586865E860400081BED7DCF
:1018D0006069B0E0319D591742F7E9E5645E640440
:1018E00000081BED7D6069B150319D591742C56BF1
:1018F00016965E960400081BED7D6069B600319D6A
:10190000591742B78B77325E320400081BED7D60B9
:1019100069B8F0319D591742E89B2DD95ED9040072
:10192000081BED7D6069BCA0319D59174261685765
:101930008D5E8D0400081BED7D6069BCC0319D5932
:1019400017427B354DB05EB00400081BED7D606929
:10195000BE60319D591742BE0C983B5E3B040008A7
:101960001BED7D6069BEA0319D591742A6EE8C1516
:101970005E150400081BED7D6069C6D0319D5917C6
:1019800042CE93880C5E0C0400081BED7D6069CB91
:1019900050319D591742CFF8CBA85EA80400081B10
:1019A000ED7D6069CE10319D591742294999E85E55
:1019B000E80400081BED7D6069CE20319D59174277
:1019C00045A366A15EA10400081BED7D6069D1807E
:1019D000319D5917427CA317565E560400081BED33
:1019E0007D6069D190319D591742AFC0C9285E28EA
:1019F0000400081BED7D6069D480319D5917428C2D
:101A0000B7AE0E5E0E0400081BED7D6069D4903108
:101A10009D59174264FE58495E490400081BED7D3C
:101A20006069D620319D5917423AAF4EE25EE2041A
:101A300000081BED7D6069D980319D5917422A79D4
:101A40005C995E990400081BED7D6069D990319D19
:101A5000591742720644B65EB60400081BED7D605D
:101A600069DD90319D5917423D3EB1305E30040032
:101A7000081BED7D6069DDD0319D591742FA099947
:101A8000A85EA80400081BED7D6069DF30319D5918
:101A9000174247A3FB3F5E3F0400081BED7D6069D2
:101AA000DF40319D5917429835E5185E180400084B
:101AB0001BED7D6069E5D0319D5917422E7848E4D1
:101AC0005EE40400081BED7D6069E5E0319D591777
:101AD00042207F30A55EA50400081BED7D6069ED06
:101AE00080319D59174243002BCA5ECA0400081B6F
:101AF000ED7D6069ED90319D59174275E44F6C5E44
:101B00006C0400081BED7D606A0A40319D59174244
:101B1000A11F1D255E250400081BED7D606A0CD009
:101B2000319D5917423C12BE805E800400081BEDB7
:101B30007D606A0D30319D591742C558771B5E1B79
:101B40000400115B0C41805097503A50A11742FDA0
:101B50006E6C945E940400115B0C418050AB40436A
:101B600050A11742911FC4745E740400115B0C29CC
:101B7000805241603850B5174278C8BFFE5EFE04FF
:101B800000215A8B4D60610BA0314689174259657F
:101B9000E6835E830400A40FF66E1B0EF722090095
:101BA000F5501200081BED7D606786F02FA0DD1652
:101BB0005A7731ABDC5EDC0400081BED7D60678783
:101BC000102FA0DD165A1C1F5C8F5E8F0400081BAF
:101BD000ED7D606789D02FA0DD165A29C941BF5E0F
:101BE000BF0400081BED7D60678E502FA0DD165AE4
:101BF0000F07E2735E730400081BED7D6067914080
:101C00002FA0DD165A314ADB365E360400081BED84
:101C10007D606798C02FA0DD165A9AB082B75EB774
:101C20000400081BED7D606799002FA0DD165AE4C3
:101C300050553F5E3F0400081BED7D60679AD02F32
:101C4000A0DD165A729A38DD5EDD0400081BED7DBA
:101C500060679DC02FA0DD165A860E2CBE5EBE04A6
:101C600000081BED7D60679DD02FA0DD165A64BE75
:101C700048985E980400081BED7D60679E202FA0A9
:101C8000DD165A504849A85EA80400081BED7D6087
:101C900067A2002FA0DD165A3E12ED245E24040038
:101CA000081BED7D6067A2202FA0DD165A73D34775
:101CB000225E220400081BED7D6067A5402FA0DD99
:101CC000165AD564D1C25EC20400081BED7D606760
:101CD000AA802FA0DD165AFC001A8B5E8B04000828
:101CE0001BED7D6067AD902FA0DD165A49F681444B
:101CF0005E440400081BED7D6067B1B02FA0DD16C7
:101D00005A3168ABB45EB40400081BED7D6067B166
:101D1000C02FA0DD165A70BDDD265E260400081B0C
:101D2000ED7D6067B6502FA0DD165AE5DBA43B5E63
:101D30003B0400081BED7D6067BCF02FA0DD165A48
:101D4000B2419D655E650400081BED7D6067BD10B6
:101D50002FA0DD165A7C5057915E910400081BEDB0
:101D60007D6067BD202FA0DD165A77AA898E5E8E12
:101D70000400081BED7D6067BEB02FA0DD165A99E8
:101D800013B97A5E7A0400081BED7D6067C3302FBB
:101D9000A0DD165A09C10E725E720400081BED7DAB
:101DA0006067C5902FA0DD165A071DA2AA5EAA047F
:101DB00000081BED7D6067C5A02FA0DD165A3F0F00
:101DC000899B5E9B0400081BED7D6067C5E02FA02A
:101DD000DD165A03E4BD385E380400081BED7D6053
:101DE00067C8C02FA0DD165AE1476E875E870400E2
:101DF000081BED7D6067CB002FA0DD165A0E6DBE6F
:101E0000515E510400081BED7D6067CB302FA0DDD3
:101E1000165A8D7BE2A85EA80400081BED7D606762
:101E2000D1202FA0DD165AFE227B115E110400087E
:101E30001BED7D6067D1302FA0DD165A0FF0A3FA9D
:101E40005EFA0400081BED7D6067D4502FA0DD16FC
:101E50005A8FBB10E75EE70400081BED7D6067D872
:101E6000102FA0DD165A2612FA415E410400081B0D
:101E7000ED7D6067DA102FA0DD165ACF37C8BD5E42
:101E8000BD0400081BED7D6067DA302FA0DD165A17
:101E9000AA6BE38F5E8F0400081BED7D6067DDE0B9
:101EA0002FA0DD165A098175875E870400081BED97
:101EB0007D6067DE102FA0DD165AFC0C235A5E5A97
:101EC0000400081BED7D6067E4A02FA0DD165AEE2C
:101ED0003CBF6E5E6E0400081BED7D6067E5102F51
:101EE000A0DD165A7969C86A5E6A0400081BED7D98
:101EF0006067E8202FA0DD165A67DB76455E450453
:101F000000081BED7D6067E8402FA0DD165A7E2596
:101F1000B7035E030400081BED7D6067E8802FA017
:101F2000DD165A9C908CAF5EAF0400081BED7D60FF
:101F300067E8902FA0DD165A5F17C9BE5EBE040089
:101F4000081BED7D6067EA602FA0DD165A622A6EDD
:101F5000EB5EEB0400081BED7D606801302FA0DD17
:101F6000165A0FB510D35ED30400081BED7D6068D0
:101F700006202FA0DD165AD98733035E030400081C
:101F80001BED7D606806302FA0DD165A324B787F3E
:101F90005E7F0400081BED7D606806602FA0DD16E3
:101FA0005A7000BAE45EE40400081BED7D606841ED
:101FB000402FA0DD165A2C54AF9E5E9E0400115B8C
:101FC0006C4D8007D5043B5F99165AB84C44E15ECE
:101FD000E10400115B6C498007D680395F9D165A79
:101FE000A2C07FC95EC90400115B6C498007D8504C
:101FF000355F9D165AA2B8879B5E9B0400215A6BE1
:1020000049609688B4314401165A05EE8D105E1071
:102010000400200FF66E200EF7220900F550120082
:10202000081BCD79604BACC0316FCD165E049A3879
:102030004A5E4A0400081BCD79604BAE60316FCD1B
:10204000165EFD1C56F95EF90400081BCD79604B45
:10205000AE70316FCD165E08EADD615E6104000886
:102060001BCD79604BAE80316FCD165E39EA9FE2B1
:102070005EE20400081BCD79604BB1C0316FCD1614
:102080005E8E5CDAF95EF90400081BCD79604BB115
:10209000D0316FCD165E927BDAD25ED20400081B7F
:1020A000CD79604BB840316FCD165EDB549E695ED2
:1020B000690400081BCD79604BB860316FCD165EA6
:1020C0002F9394705E700400081BCD79604BBD9017
:1020D000316FCD165E5A3E5B925E920400081BCDB6
:1020E00079604BBDA0316FCD165EF6A56FA15EA1E4
:1020F0000400081BCD79604BD4C0316FCD165EACA7
:10210000529FF55EF50400081BCD79604BD6B031C7
:102110006FCD165E00191EE15EE10400081BCD794B
:10212000604BD6D0316FCD165E7C6145DE5EDE043D
:1021300000081BCD79604BDAA0316FCD165E1521FA
:102140007DB35EB30400081BCD79604BDAF0316FCC
:10215000CD165EB64D54055E050400081BCD7960B2
:102160004BDDD0316FCD165E3FB376775E770400DE
:10217000081BCD79604BE1E0316FCD165E82FC9A91
:10218000655E650400081BCD79604BE960316FCD59
:10219000165EA9C65D3B5E3B0400081BCD79604B13
:1021A000E970316FCD165E3BDCE8165E1604000860
:1021B0001BCD79604BE9B0316FCD165E541E44D70C
:1021C0005ED70400081BCD79604C1A90316FCD1694
:1021D0005E624ACCE95EE90400081BCD79604C1AC6
:1021E000A0316FCD165ED3659D165E160400081BE8
:1021F000CD79604C2200316FCD165E023F00985EB3
:10220000980400081BCD79604C2480316FCD165E98
:10221000F627DB295E290400081BCD79604C24C019
:10222000316FCD165EF01075F65EF60400081BCD1A
:1022300079604C2980316FCD165EDC3E09C55EC5E4
:102240000400081BCD79604C2EE0316FCD165E2462
:102250007A46515E510400081BCD79604C2F003145
:102260006FCD165E704FEB7C5E7C0400081BCD7951
:10227000604C3160316FCD165E591298055E0504D1
:1022800000081BCD79604C3180316FCD165E271F61
:10229000ABA55EA50400081BCD79604C3590316F6D
:1022A000CD165EF34591055E050400081BCD7960EF
:1022B0004C36F0316FCD165E28EB6BE95EE9040019
:1022C000081BCD79604C3700316FCD165E4A00B5E2
:1022D0004F5E4F0400081BCD79604C3710316FCD35
:1022E000165EBFDB25E15EE10400081BCD79604C82
:1022F0003730316FCD165E15D097D25ED20400080C
:102300001BCD79604C3740316FCD165E7E91D3CCBA
:102310005ECC0400081BCD79604C3990316FCD162E
:102320005EFF3662855E850400081BCD79604C39FE
:10233000D0316FCD165EAC3C33CD5ECD0400081BB2
:10234000CD79604C3E80316FCD165EAF3FE0495E87
:10235000490400081BCD79604C4C70316FCD165E7E
:1023600048B7D2965E960400081BCD79604C4E505B
:10237000316FCD165E00CD673F5E3F0800081BCD74
:1023800079604C55D0316FCD165E3D494F395E397D
:102390000400081BCD79604C5620316FCD165EB914
:1023A0001E25735E730400081BCD79604C71E0310B
:1023B0006FCD165E7001D4B35EB30400081BCD79F7
:1023C000604C79A0316FCD165E112FCEAE5EAE049B
:1023D00000081BCD79604C7C20316FCD165ECF623A
:1023E00090E65EE60400081BCD79604C7C50316FAE
:1023F000CD165EBE3F59735E730400081BCD796035
:102400004C7C80316FCD165EF961C1225E220400E2
:10241000081BCD79604C80B0316FCD165E65499F49
:10242000045E040400081BCD79604C8100316FCD3F
:10243000165E4676192F5E2F0400215A8B4D60726E
:1024400003743646C9165E3D68278C5E8C04001105
:102450005AEC4180A02450315095165EDC32B48392
:102460005E830400115AEC4180A024D4425095169A
:102470005EC584513E5E3E0400002563315D2052FE
:102480006573657420284D6167656E74612920202D
:10249000202020202020202020202020202020203C
:1024A000325D20526573657420284C69676874201A
:1024B0004D6167656E746129202020202020202036
:1024C00025630D0A00002563335D20526573657432
:1024D000202850686F746F20426C61636B29202044
:1024E000202020202020202020202020345D205269
:1024F0006573657420284D6174746520426C616356
:102500006B292020202020202020202025630D0A58
:1025100000002563355D2052657365742028596578
:102520006C6C6F7729202020202020202020202064
:102530002020202020202020365D205265736574E5
:1025400020284C69676874204379616E2920202017
:10255000202020202020202025630D0A0000256354
:10256000375D20526573657420284C696768742054
:10257000477261792920202020202020202020203F
:1025800020202020385D205265736574202843790F
:10259000616E2920202020202020202020202020A3
:1025A0002020202025630D0A000025633D3D3D3D90
:1025B0003D3D3D3D3D3D3D3D3D3D3D3D3D3D3D3D4B
:1025C0003D3D3D3D3D3D3D3D3D3D3D3D3D3D3D3D3B
:1025D0003D3D3D3D3D3D3D3D3D3D3D3D3D3D3D3D2B
:1025E0003D3D3D3D3D3D3D3D3D3D3D3D3D3D3D3D1B
:1025F00025630D0A00002563415D2052656164205A
:10260000636869702064617461202020202020208C
:10261000202020202020202020202020465D204433
:102620006973706C61792043726564697473207397
:1026300074617475732020202020202025630D0AEA
:1026400000002563475D20526563686172676520FD
:102650004372656469747320636F756E746572206C
:102660002020202020202020485D205669657720EA
:1026700063686970206669726D7761726520726542
:102680006C6561736520202025630D0A00002563B9
:10269000495D20536574206D616E75666163747564
:1026A0007265206461746520202020202020202075
:1026B00020202020455D20546F67676C65204465AD
:1026C00076656C6F706D656E74204D6F646520204B
:1026D0002020202025630D0A00002563435D205340
:1026E000657420636869702073657269616C206E1F
:1026F000756D6265722873746172742920202020C0
:102700004A5D2050726F6772616D20496E6B206464
:1027100061746520746F2063686970202020202018
:1027200025630D0A00002563425D205772697465B8
:10273000206461746120696E746F20636869702819
:10274000312062797465292020202020595D205293
:102750006561642063686970206461746128756EC6
:10276000666F726D617474656429202025630D0A9B
:10277000000025634B5D20436F70792063686970AA
:10278000206461746120202020202020202020202F
:1027900020202020202020204C5D20506173746573
:1027A00020636869702064617461202020202020EB
:1027B000202020202020202025630D0A00002563F2
:1027C0004D5D205669657720636869702073657276
:1027D00069616C206E756D6265722020202020205A
:1027E000202020204E5D205669657720636869703F
:1027F000206D616E756661637475726520646174C5
:102800006520202025630D0A00002563515D2056B8
:10281000696577206368697020696E6B206C6576E6
:10282000656C202020202020202020202020202017
:10283000525D20526563616C6962726174652063E8
:10284000686970206461746120286D616E2E292092
:1028500025630D0A000020233931204D6167656E24
:102860007461202843393436384129202020202023
:102870002020200020233931204C69676874204DC6
:102880006167656E746120284339343731412920EE
:102890002000202339312050686F746F20426C6112
:1028A000636B20284339343635412920202020000D
:1028B00020233931204D6174746520426C61636B53
:1028C0002028433934363541292020202000202378
:1028D00039312059656C6C6F77202843393436398B
:1028E00041292020202020202020200020233931B1
:1028F000204C69676874204379616E20284339341D
:102900003730412920202020200020233931204C3D
:1029100069676874204772617920284339343636F4
:1029200041292020202020002023393120437961B3
:102930006E20284339343638412920202020202099
:102940002020202020000D0A0A43415554494F4EB3
:10295000202D2053657269616C206E756D62657201
:102960002070726F6772616D6D696E672066616954
:102970006C65642E2054727920616761696E212133
:1029800025632000373735206D6C0D0A0000343088
:1029900030206D6C0D0A0000556E6B6E6F776E0DFA
:1029A0000A004A616E756172792020004665627284
:1029B0007561727920004D617263682020202000CB
:1029C000417072696C20202020004D617920202008
:1029D000202020004A756E652020202020004A75A6
:1029E0006C792020202020004175677573742020A9
:1029F000200053657074656D626572004F63746F7B
:102A00006265722020004E6F76656D6265722000EF
:102A1000446563656D6265722000494E4B4A4554BA
:102A20002053595354454D5320507479284C5444E5
:102A3000290053696E6761706F7265002B2B363504
:102A40002E363333332D3333303200002020202014
:102A500020202020207777772E73616D2D696E6B93
:102A60002E636F6D0000202D20446576696365201C
:102A70006661696C656420746F2041434B000D0AE8
:102A8000436869702073657269616C206E756D6250
:102A900065723A20000043617061636974793A207D
:102AA0000000496E6B206C6576656C3A2000256CE1
:102AB00075206D6C0D0A00000D0A0A436F6E74726A
:102AC0006F6C204279746520577269746520737544
:102AD000636365737366756C00000D0A0A436F6E5D
:102AE00074726F6C20427974652057726974652026
:102AF000776173206E6F742073756363657373669B
:102B0000756C00000D0A0A535020577269746520D5
:102B10007375636365737366756C00000D0A0A5301
:102B20005020577269746520776173206E6F74202E
:102B30007375636365737366756C00000D0A456E8B
:102B400074657220746865206164647265737320B3
:102B5000746F20726561642066726F6D2E2E3A204C
:102B600000000D0A456E7465722074686520484542
:102B700058206164647265737320746F2077726982
:102B8000746520746F2E2E3A20000D0A456E746510
:102B900072204845582062797465204E6F2E254476
:102BA00020746F206265207772697474656E3A20B4
:102BB00000000D0A507265737320616E79206B6599
:102BC0007920746F20636F6E74696E75652E2E2E7A
:102BD00000000D0A0A4552524F52202D20546865BC
:102BE00020536372617463687061642077726974E2
:102BF00065206661696C656400000D0A0A455252E1
:102C00004F52202D20436F756C64206E6F742075B9
:102C1000706461746520746865206E6577206368F0
:102C200065636B73756D20402061646472657373B6
:102C30002030783739002020202A2A2A2A20476588
:102C40006E6572696320485020444A5A36313030EC
:102C500020496E6B204368697020526573657474F7
:102C600065722056657220312E323420436F7079A0
:102C7000726967687428432932303130202A2A2A41
:102C80002A0D0A00202020202020202020200000C3
:102C9000202D2054656C3A00202020202020202068
:102CA000202020202020000020202020202025631C
:102CB00000002020202020202563204D61696E2007
:102CC0004D656E75202D20002A2A2A204E6F207611
:102CD000616C69642063686970207965742065732C
:102CE0007461626C6973686564202A2A2A20202036
:102CF0002020202025630D0A000023393120506850
:102D00006F746F20426C61636B203737356D6C20B8
:102D10002843393436354129202000002339312019
:102D20004C69676874204379616E203737356D6C64
:102D3000202843393437304129202020000023390E
:102D400031204C69676874204D6167656E7461203D
:102D50003737356D6C20284339343731412900002D
:102D6000233931204C6967687420477261792037B4
:102D700037356D6C202843393436364129202020E0
:102D80000000233931204D6174746520426C616309
:102D90006B203737356D6C20284339343634412960
:102DA00020200000233931204379616E20373735E8
:102DB0006D6C2028433934363841292020202020CA
:102DC000202020200000233931204D6167656E747A
:102DD00061203737356D6C20284339343638412926
:102DE00020202020202000002339312059656C6CE0
:102DF0006F77203737356D6C2028433934363941A9
:102E000029202020202020200000556E6B6E6F7737
:102E10006E2044657669636520307825325820201D
:102E200020202020202020202020200020202020C2
:102E3000202020202020202025430D0A00000D0AFC
:102E400053656C656374206F7074696F6E3A2020EF
:102E500000000D0A436865636B73756D2028307838
:102E600037412920636F72726563746564202D2079
:102E700077617320253258202D206E65772025320A
:102E8000580A00000D0A436865636B73756D20284E
:102E9000307837412920546573746564204F4B0A9C
:102EA00000004465766963652053657269616C2032
:102EB0004E756D6265723A256C75202D20526573D2
:102EC0006574206C6F673A25750D0A0A000028505A
:102ED0006C65617365204E4F54453A2074686520D7
:102EE00061626F766520696E666F726D6174696F7D
:102EF0006E206D7573742062652071756F746564E2
:102F0000207768656E2070757263686173696E679B
:102F100020637265646974732E0D0A0054686973C6
:102F200020696E666F726D6174696F6E20697320BF
:102F30007573656420746F2067656E657261746572
:102F40002061206B657920746861742077696C6CEE
:102F50002062652073656E74206261636B20746FFC
:102F600020796F752E290D0A0A0043726564697411
:102F7000732072656D61696E696E673A20256C75A4
:102F80000D0A0A000D0A456E74657220746865208A
:102F90006E756D626572206F662072657365742050
:102FA00063726564697473206265696E6720707509
:102FB000726368617365643A2D2020000D0A456EC6
:102FC00074657220746865203430206368617261B2
:102FD00063746572206B6579636F646520737570C7
:102FE000706C69656420627920003A2D200D0A001A
:102FF0000D0A526573657420637265646974732089
:10300000616D6D656E64656420737563636573736C
:1030100066756C6C792066726F6D20256C752074F6
:103020006F20256C752E00000D0A496E76616C6963
:103030006420636F64652E002A2A2A2A0000522029
:103040004520532045205400572052204920542029
:103050004520202020502052204F2043204520533F
:10306000205300002020205320552043204320459A
:10307000205320462055204C2A2A2A2A00000A0ADA
:103080000D524553455420636F756E746572206907
:10309000732061646A757374656420746F3A2025C7
:1030A0006C750A0D00000D0A20284E6F20637265B2
:1030B000646974732072656D61696E696E672E2034
:1030C00050757263686173652063726564697473B7
:1030D0002066726F6D2046542E290D0A0000284389
:1030E000415554494F4E2120596F752068617665CE
:1030F00020256C75206372656469740020617661B7
:10310000696C61626C652E205075726368617365CD
:1031100020637265646974732066726F6D200000AD
:103120002E290D0A0000080E016E050E006E002EFD
:10313000FED78B969496060E006E002EFED70101E8
:1031400027378B98D8B09488D8A09498948682A674
:10315000FED7012E01D002D00001E7D7050E006E88
:10316000002EFED78B96949600009488060E006E73
:10317000002EFED7060E006E002EFED7948682A685
:10318000FED7016A060E006E002EFED782B80180BF
:103190008B9694968B9894980001000C01012681DF
:1031A0009488050E006E002EFED79486060E006EE3
:1031B000002EFED78B989498050E006E002EFED739
:1031C0008B96949625C127F10001ADDF01500101D6
:1031D000269101B0268194980000948682A6FED79D
:1031E000050E006E002EFED700D000009488050E5C
:1031F000006E002EFED7000E26A1010E016E00010A
:1032000096EF1DF01B0E04009EA8FDD7AD6E5B0E61
:1032100004009EA8FDD7AD6E320E04009EA8FDD717
:10322000AD6E4A0E04009EA8FDD7AD6E000C0101E4
:103230002C51016A2B5D03E22BC100F00CD0006A17
:10324000080E2D6F2B3700362C51005CD8B0006E65
:1032500001362D2FF7D70001000C015029C12BF1A9
:10326000640E01012C6F0001E2DF00C029F1015062
:10327000300E08E101012AA30FD02AB70DD02AB9D8
:10328000200E04D001012A972A992A810126015093
:1032900004009EA8FDD7AD6E29C12BF10A0E2C6F3C
:1032A0000001C5DF00C029F10150300E08E1010125
:1032B0002AB70CD02AA10AD02AB9200E0001012673
:1032C000015004009EA8FDD7AD6E0101300E2927E4
:1032D000295104009EA8FDD7AD6E0001000C1B0E05
:1032E00004009EA8FDD7AD6E5B0E04009EA8FDD71E
:1032F000AD6E26C129F11B0E01012A6F0001ADDF61
:103300003B0E04009EA8FDD7AD6E27C129F11B0E10
:1033100001012A6F0001A1DF3B0E04009EA8FDD72A
:10332000AD6E28C129F11B0E01012A6F000195DF46
:103330006D0E04009EA8FDD7AD6E000C0900F5527D
:103340000EE0F6CF26F1F7CF27F1F55004009EA846
:10335000FDD7AD6E26C1F6FF27C1F7FFEFD7000CF2
:103360001B0E04009EA8FDD7AD6E5B0E04009EA848
:10337000FDD7AD6E0101296B1B0E2A6F00016DDFB9
:103380003B0E04009EA8FDD7AD6E3B0E04009EA828
:10339000FDD7AD6E6D0E04009EA8FDD7AD6E000C7E
:1033A000010E0101266F250E276F280E286F0001E0
:1033B00096DF360EF66E2C0EF76EC0DF840EF66EBC
:1033C0002C0EF76EBBDF1A0EF66E2A0EF76EB6DF06
:1033D0002E0E04009EA8FDD7AD6E200E04009EA800
:1033E000FDD7AD6E320EF66E2A0EF76EA7DF900E89
:1033F000F66E2C0EF76EA2DF3C0EF66E2A0EF76EFE
:103400009DDF2E0E04009EA8FDD7AD6E0D0E0400AC
:103410009EA8FDD7AD6E0A0E04009EA8FDD7AD6E26
:10342000980EF66E2C0EF76E89DF4C0EF66E2A0E95
:10343000F76E84DF0D0E04009EA8FDD7AD6E0A0E58
:1034400004009EA8FDD7AD6E0D0E04009EA8FDD70A
:10345000AD6E0A0E04009EA8FDD7AD6E81DF000C94
:103460000900F6CF27F1F7CF28F1F55004009EA808
:10347000FDD7AD6E27C1F6FF28C1F7FF0101262F4A
:1034800001D002D00001ECD70001000C010127BFE0
:1034900011D00F0E006E263900160A0E005C03E2F2
:1034A000300E002602D027510026005004009EA8AE
:1034B000FDD7AD6E0F0E26170A0E265D02E2300E06
:1034C00002D0279F27512627265104009EA8FDD70A
:1034D000AD6E0001000C0D0E04009EA8FDD7AD6E70
:1034E0000A0E04009EA8FDD7AD6EA80EF66E2C0E37
:1034F000F76E060E0101266F0001B2DFC90E04004F
:103500009EA8FDD7AD6E0101256B2551380807E354
:10351000CD0E04009EA8FDD7AD6E252BF6D7BB0EB1
:1035200004009EA8FDD7AD6E0D0E04009EA8FDD729
:10353000AD6E0A0E04009EA8FDD7AD6EB20EF66EFB
:103540002C0EF76E060E266F00018ADFBA0E0400FD
:103550009EA8FDD7AD6EBA0EF66E2C0EF76E0D0E50
:103560000101266F00017CDF1A5219E1C80EF66EC8
:103570002C0EF76E2C0E0101266F000171DFBA0EC2
:1035800004009EA8FDD7AD6E0D0E04009EA8FDD7C9
:10359000AD6E0A0E04009EA8FDD7AD6EBED01A50C7
:1035A000B10A10E0020A1DE0060A2AE0020A37E02A
:1035B0000E0A44E0020A51E0060A5EE0020AD8B4AC
:1035C0006AD078D0010E0101266F1E0E276F2F0ED4
:1035D000286F000184DEFA0EF66E2C0EF76EAEDE5A
:1035E00083D0020E0101266F240E276F280E286F4C
:1035F000000175DE1C0EF66E2D0EF76E9FDE74D088
:10360000020E0101266F230E276F280E286F00017E
:1036100066DE3E0EF66E2D0EF76E90DE65D0020E63
:103620000101266F1E0E276F2F0E286F000157DE37
:10363000600EF66E2D0EF76E81DE56D0010E010182
:10364000266F1E0E276F2F0E286F000148DE820E98
:10365000F66E2D0EF76E72DE47D0010E0101266F59
:10366000240E276F280E286F000139DEA40EF66E97
:103670002D0EF76E63DE38D0010E0101266F230E8A
:10368000276F280E286F00012ADEC60EF66E2D0E5B
:10369000F76E54DE29D0010E0101266F210E276F2F
:1036A000280E286F00011BDEE80EF66E2D0EF76E59
:1036B00045DE1AD00A0EF66E2E0EF76E110E0101BF
:1036C000266F0001CDDE1AC026F1370E0101276FEB
:1036D0000001DCDE1E0EF66E2E0EF76E0D0E0101E1
:1036E000266F0001BDDE00D03BDE2C0EF66E2E0EE6
:1036F000F76E0C0E0101266F0001B2DEBA0E040057
:103700009EA8FDD7AD6E0D0E04009EA8FDD7AD6E30
:103710000A0E04009EA8FDD7AD6EDA0E04009EA826
:10372000FDD7AD6EC40E04009EA8FDD7AD6EC40ECD
:1037300004009EA8FDD7AD6EC40E04009EA8FDD760
:10374000AD6EC40E04009EA8FDD7AD6EC40E04007D
:103750009EA8FDD7AD6ED00E04009EA8FDD7AD6E1D
:103760000101256B2551380807E3C40E04009EA80B
:10377000FDD7AD6E252BF6D7D00E04009EA8FDD741
:10378000AD6EC40E04009EA8FDD7AD6EC40E04003D
:103790009EA8FDD7AD6EC40E04009EA8FDD7AD6EE9
:1037A000C40E04009EA8FDD7AD6EBF0E04009EA8F7
:1037B000FDD7AD6E0D0E04009EA8FDD7AD6E0A0EAE
:1037C00004009EA8FDD7AD6EB30E04009EA8FDD7E1
:1037D000AD6E7C0EF66E240EF76E440E266F000161
:1037E0003FDEB30E04009EA8FDD7AD6E0D0E0400A3
:1037F0009EA8FDD7AD6E0A0E04009EA8FDD7AD6E43
:10380000B30E04009EA8FDD7AD6EC80EF66E240E52
:10381000F76E440E0101266F000122DEB30E040094
:103820009EA8FDD7AD6E0D0E04009EA8FDD7AD6E0F
:103830000A0E04009EA8FDD7AD6EB30E04009EA82C
:10384000FDD7AD6E140EF66E250EF76E440E010117
:10385000266F000105DEB30E04009EA8FDD7AD6EF5
:103860000D0E04009EA8FDD7AD6E0A0E04009EA8A2
:10387000FDD7AD6EB30E04009EA8FDD7AD6E600EF1
:10388000F66E250EF76E440E0101266F0001E8DD8D
:10389000B30E04009EA8FDD7AD6E0D0E04009EA8C9
:1038A000FDD7AD6E0A0E04009EA8FDD7AD6EB30E17
:1038B00004009EA8FDD7AD6EAC0EF66E250EF76E19
:1038C000440E0101266F0001CBDDB30E04009EA85B
:1038D000FDD7AD6E0D0E04009EA8FDD7AD6E0A0E8D
:1038E00004009EA8FDD7AD6EB30E04009EA8FDD7C0
:1038F000AD6EF80EF66E250EF76E440E0101266FC2
:103900000001AEDDB30E04009EA8FDD7AD6E0D0E16
:1039100004009EA8FDD7AD6E0A0E04009EA8FDD738
:10392000AD6EB30E04009EA8FDD7AD6E440EF66ECC
:10393000260EF76E440E0101266F000191DDB30ED5
:1039400004009EA8FDD7AD6E0D0E04009EA8FDD705
:10395000AD6E0A0E04009EA8FDD7AD6EB30E040036
:103960009EA8FDD7AD6E900EF66E260EF76E440E35
:103970000101266F000174DDB30E04009EA8FDD77F
:10398000AD6E0D0E04009EA8FDD7AD6E0A0E0400AC
:103990009EA8FDD7AD6EB30E04009EA8FDD7AD6EF8
:1039A000DC0EF66E260EF76E440E0101266F000146
:1039B00057DDB30E04009EA8FDD7AD6E0D0E0400BA
:1039C0009EA8FDD7AD6E0A0E04009EA8FDD7AD6E71
:1039D0009CA31DD0B30E04009EA8FDD7AD6E280E8B
:1039E000F66E270EF76E440E0101266F000138DDDA
:1039F000B30E04009EA8FDD7AD6E0D0E04009EA868
:103A0000FDD7AD6E0A0E04009EA8FDD7AD6EB30EB5
:103A100004009EA8FDD7AD6E740EF66E270EF76EED
:103A2000440E0101266F00011BDDB30E04009EA8A9
:103A3000FDD7AD6E0D0E04009EA8FDD7AD6E0A0E2B
:103A400004009EA8FDD7AD6EB30E04009EA8FDD75E
:103A5000AD6EC00EF66E270EF76E440E0101266F96
:103A60000001FEDCB30E04009EA8FDD7AD6E0D0E66
:103A700004009EA8FDD7AD6E0A0E04009EA8FDD7D7
:103A8000AD6EB30E04009EA8FDD7AD6E0C0EF66EA3
:103A9000280EF76E440E0101266F0001E1DCB30E23
:103AA00004009EA8FDD7AD6E0D0E04009EA8FDD7A4
:103AB000AD6E0A0E04009EA8FDD7AD6EC00E0400C8
:103AC0009EA8FDD7AD6E0101256B2551430807E384
:103AD000C40E04009EA8FDD7AD6E252BF6D7D90ED7
:103AE00004009EA8FDD7AD6E0D0E04009EA8FDD764
:103AF000AD6E0A0E04009EA8FDD7AD6E0001000C4D
:103B000002EC19F04DDCE7DC3E0EF66E2E0EF76E81
:103B100015DC000CD190B10E0101246F2451BF08B7
:103B20001CE324C125F10001CEEF18F0015211E091
:103B30001A500101245D0AE024C11AF00001E0DFFF
:103B40001AC01BF0D18015D004D00101D180000132
:103B500010D0020E01012427E1D704001A6A1B507D
:103B60001A5C05E00001CCDF1AC01BF00101D18016
:103B70000001F29430EF00F00D0A202020203030B8
:103B80002030312030322030332030342030352086
:103B90003036203037203038203039203041203046
:103BA000422030432030442030452030460D0A006A
:103BB0000D0A4E4F54453A2D2054686520646574B3
:103BC00065637465642063686970206973206E6F33
:103BD000742066726F6D2074686520444A343030FA
:103BE000302066616D696C792E2054727920616E87
:103BF0006F746865722E0D0A00000D0A5468652006
:103C000074656D706C6174652064617461207265A7
:103C100070726573656E74732061200020496E7642
:103C2000616C696420646174610D0A000D0A0A57B1
:103C300072697465207375636365737366756C0070
:103C40000D0A0A5772697465206E6F74207375636C
:103C50006365737366756C2057726974653A2532B3
:103C60005820526561643A25325800000D0A0A4313
:103C7000415554494F4E202D204352432070726FBE
:103C80006772616D6D696E67206661696C6564203D
:103C90006174206164647265737320307837412EDB
:103CA0002054727920616761696E6E2121000D0ACE
:103CB0000A43415554494F4E202D20435243207012
:103CC000726F6772616D6D696E67206661696C65A0
:103CD0006420617420616464726573732030783786
:103CE000442E2054727920616761696E6E21210033
:103CF0000D0A0A53657269616C206E756D6265729A
:103D00002070726F6772616D6D6564207375636397
:103D100065737366756C6C79212120000D0A0A4366
:103D2000757272656E742043726564697473206184
:103D30007661696C6162653A20256C750A0D000038
:103D40002A2A2A2A52204520532045205420202068
:103D50005320552043204320452053204620552002
:103D60004C2A2A2A2A000A0A0D5245534554206338
:103D70006F756E7465722069732061646A757374FF
:103D8000656420746F3A20256C750A0D00000A0DD9
:103D90004669726D77617265205265766973696FE5
:103DA0006E3A2D2532582E2532583A0A0D000D0A4A
:103DB000496E707574206465766963652079656104
:103DC00072283230303720746872752032303137C3
:103DD000293A20000D0A496E707574206465766971
:103DE0006365206D6F6E7468283120746872752069
:103DF000313229203A2000000D0A496E7075742076
:103E0000646576696365206461792831207468721D
:103E10007520333129203A2000000D0A4465766967
:103E200063652064617465207265636F72646564A4
:103E3000207375636365737366756C6C792E0D0AF8
:103E4000000050726F6772616D6D65642063686910
:103E500070732077696C6C206E6F7720636F6E745F
:103E600061696E207468697320656E636F64656450
:103E700020646174652076616C75652E202575203F
:103E800000005468652052657365742F5061737427
:103E900065206F7065726174696F6E207761732041
:103EA0004E4F54207375636365737366756C21217F
:103EB00000000A0D416464726573733A253258201C
:103EC000446174613A2532580A0D0000496E7075DC
:103ED0007420646576696365207965617228323083
:103EE000303720746872752032303137293A20001B
:103EF0000D0A496E70757420646576696365206D7E
:103F00006F6E7468283120746872752031322920F0
:103F10003A2000000D0A496E707574206465766958
:103F200063652064617928312074687275203331AB
:103F300029203A2000000D0A4461746520636861FD
:103F40006E6765207375636365737366756C6C2E3D
:103F50000D0A000050726F6772616D6D65642063B9
:103F6000686970732077696C6C206E6F7720636F5F
:103F70006E7461696E207468697320656E636F6426
:103F8000656420646174652076616C75652E2025FA
:103F900032582532580D0A004368697020636F70EB
:103FA0007920636F6D706C657465642073756363ED
:103FB00065737366756C6C792121000044617461CE
:103FC00020636F7079206661696C6564202D2074B0
:103FD000727920616761696E21210D0A0A004164CE
:103FE000647220253258203A2052656164202532BF
:103FF00058202D20436F7272656374204461746190
:1040000020253258000092908990000CEA6AD10E67
:10401000E96EEF5011E0060E016EBF0E006E040057
:10402000002EFDD7012EF9D77A0E006E002EFED796
:1040300000D00400EF2EEFD7000C9486948890EF08
:104040003FF01B0E04009EA8FDD7AD6E630E04006A
:104050009EA8FDD7AD6E92EF3FF0196AF2BE198EA1
:10406000F29E020E0101266F250E276F280E286F83
:1040700000016FEC19F019BEF28EB86BB851180838
:104080000DE3B96BB9514F0807E3200E04009EA859
:10409000FDD7AD6EB92BF6D7B82BF0D7196AF2BEA3
:1040A000198EF29EB0EC19F019BEF28E94EF3FF02B
:1040B0009488050E006E002EFED79486060E006EC4
:1040C000002EFED78B989498050E006E002EFED71A
:1040D0008B969496010E1A5CC56F196AF2BE198E02
:1040E000F29EE8CF27F193EC18F019BEF28E196A10
:1040F000F2BE198EF29EC3C027F193EC18F019BEE0
:10410000F28E196AF2BE198EF29EC4C027F193ECAA
:1041100018F019BEF28E94980000948682A6FED7FD
:10412000050E006E002EFED700D000009488050E0C
:10413000006E002EFED7000CC36BC26BC181C1A103
:104140004FD004009488050E006E002EFED7948692
:10415000060E006E002EFED78B989498050E006E0A
:10416000002EFED78B969496196AF2BE198EF29E97
:104170001AC027F193EC18F019BEF28E0150C191CC
:1041800001B0C18194980000948682A6FED7050EE6
:10419000006E002EFED700D000009488050E006E41
:1041A000002EFED7C22BD8B4C32BC351000814E293
:1041B000FF0A03E1C251F4080FE2660EF66E2A0E02
:1041C000F76E196AF2BE198EF29E9EEC19F019BEB6
:1041D000F28E000E016E06D0010ED16F17DFAFD741
:1041E000010E016E000C7C0EC36FAA0EC46F60DF5F
:1041F000000CC251C403F3CF01F0F4CF00F0C503AB
:10420000F3500026C351C403F3500020026E000C8B
:10421000080EC56F00C0C6F09488060E006E002E12
:10422000FED7948682A6FED782B8D88082A8D8907E
:104230000136050E006E002EFED794968B96C52F84
:10424000EBD79488060E006E002EFED78B98C651D1
:10425000D8A494980000948682A6FED7050E006E1E
:10426000002EFED78B969496060E006E002EFED77B
:104270008B989498000C9488050E006E002EFED743
:104280009486060E006E002EFED78B989498050E2D
:10429000006E002EFED78B969496196AF2BE198E88
:1042A000F29E1AC027F193EC18F019BEF28E196A2B
:1042B000F2BE198EF29EC2C027F193EC18F019BE1F
:1042C000F28E006AA5DF01C0C3F0949800009486C6
:1042D00082A6FED7050E006E002EFED700D000008D
:1042E0009488050E006E002EFED7C3C001F0000CAE
:1042F0008ADE800EBD5DF80FD8B021EF26F0080FE2
:1043000080EF26F0F2CFC1F0F29EAA6A300EA96EBD
:10431000A69CA69EA680A850C1BFF28EBF6FBE6BA2
:10432000BE51140865E35FDF036ABE5157EC00F02D
:10433000C16FC36BBFC0C2F0C56B150EC46F59DF30
:1043400002C0C3F001C0C2F0BE510124016E000ED4
:104350000220036E015003C0F7FF6AEC00F0C26F49
:10436000C1C0C3F0C46FA4DEE7DE036ABE5157ECE0
:1043700000F0C16FC26F7FDF01C0C0F0C36BBFC070
:10438000C2F0C56B150EC46F34DF02C0C2F001C0AD
:10439000C1F0BE510124016E000E0220036E0150D7
:1043A00003C0F7FF6AEC00F0016EC05D1FE002EC95
:1043B00019F0460EF66E290EF76E196AF2BE198EC6
:1043C000F29E3A0E0101266F000130EC1AF019BE80
:1043D000F28E070E04009EA8FDD7AD6E200E0400DD
:1043E0009EA8FDD7AD6E9C957EEF26F0BE2B98D78C
:1043F000BF2BBF51360801E2BF6BAA6A300EA96E0F
:10440000BFC0A8FFA69CA69EA684F250006EF29E96
:104410000F01550EA76EAA0EA76EA682A6B2FED7F2
:10442000A6940050F212000121EF26F0F2CFC1F065
:10443000F29EAA6A310EA96EA69CA69EA680A850DE
:10444000C1BFF28EBF6FBE6BBE51140865E3CBDEF9
:10445000036ABE5157EC00F0C16FC36BBFC0C2F01E
:10446000C56B150EC46FC5DE02C0C3F001C0C2F03B
:10447000BE510124016E000E0220036E015003C0E4
:10448000F7FFB3EC02F0C26FC1C0C3F0C46F10DE1F
:1044900053DE036ABE5157EC00F0C16FC26FEBDE12
:1044A00001C0C0F0C36BBFC0C2F0C56B150EC46FB6
:1044B000A0DE02C0C2F001C0C1F0BE510124016EF5
:1044C000000E0220036E015003C0F7FFB3EC02F0B0
:1044D000016EC05D1FE002EC19F0460EF66E290E6B
:1044E000F76E196AF2BE198EF29E3A0E0101266F1E
:1044F000000130EC1AF019BEF28E070E04009EA8DF
:10450000FDD7AD6E200E04009EA8FDD7AD6E9C9524
:104510007EEF26F0BE2B98D7BF2BBF51340801E2A7
:10452000BF6BAA6A310EA96EBFC0A8FFA69CA69E4B
:10453000A684F250006EF29E0F01550EA76EAA0ED1
:10454000A76EA682A6B2FED7A6940050F212000172
:1045500078D3F2CFC1F0F29EAA6A320EA96EA69C61
:10456000A69EA680A850C1BFF28EBF6FBE6BBE5183
:10457000140864E338DE036ABE5157EC00F0C16FE3
:10458000C36BBFC0C2F0C56B150EC46F32DE02C074
:10459000C3F001C0C2F0BE510124016E000E022022
:1045A000036E015003C0F7FFE7EC04F0C26FC1C017
:1045B000C3F0C46F7DDDC0DD036ABE5157EC00F06F
:1045C000C16FC26F58DE01C0C0F0C36BBFC0C2F084
:1045D000C56B150EC46F0DDE02C0C2F001C0C1F084
:1045E000BE510124016E000E0220036E015003C073
:1045F000F7FFE7EC04F0016EC05D1EE002EC19F07D
:10460000460EF66E290EF76E196AF2BE198EF29EEC
:104610003A0E0101266F000130EC1AF019BEF28E3D
:10462000070E04009EA8FDD7AD6E200E04009EA8C4
:10463000FDD7AD6E9C9562D3BE2B99D7BF2BBF51D2
:10464000340801E2BF6BAA6A320EA96EBFC0A8FF90
:10465000A69CA69EA684F250006EF29E0F01550EF7
:10466000A76EAA0EA76EA682A6B2FED7A694005089
:10467000F2120001E6D2F2CFC1F0F29EAA6A330E26
:10468000A96EA69CA69EA680A850C1BFF28EBF6F41
:10469000BE6BBE51140864E3A6DD036ABE5157EC3D
:1046A00000F0C16FC36BBFC0C2F0C56B150EC46F05
:1046B000A0DD02C0C3F001C0C2F0BE510124016EF2
:1046C000000E0220036E015003C0F7FF1BEC07F041
:1046D000C26FC1C0C3F0C46FEBDC2EDD036ABE51F4
:1046E00057EC00F0C16FC26FC6DD01C0C0F0C36BF4
:1046F000BFC0C2F0C56B150EC46F7BDD02C0C2F037
:1047000001C0C1F0BE510124016E000E0220036EF3
:10471000015003C0F7FF1BEC07F0016EC05D1EE007
:1047200002EC19F0460EF66E290EF76E196AF2BE0B
:10473000198EF29E3A0E0101266F000130EC1AF03C
:1047400019BEF28E070E04009EA8FDD7AD6E200E96
:1047500004009EA8FDD7AD6E9C95D0D2BE2B99D7F4
:10476000BF2BBF51350801E2BF6BAA6A330EA96E99
:10477000BFC0A8FFA69CA69EA684F250006EF29E23
:104780000F01550EA76EAA0EA76EA682A6B2FED77F
:10479000A6940050F212000154D2F2CFC1F0F29E62
:1047A000AA6A340EA96EA69CA69EA680A850C1BF78
:1047B000F28EBF6FBE6BBE51140864E314DD036A52
:1047C000BE5157EC00F0C16FC36BBFC0C2F0C56BE8
:1047D000150EC46F0EDD02C0C3F001C0C2F0BE51A1
:1047E0000124016E000E0220036E015003C0F7FF8A
:1047F00059EC09F0C26FC1C0C3F0C46F59DC9CDC36
:10480000036ABE5157EC00F0C16FC26F34DD01C0C6
:10481000C0F0C36BBFC0C2F0C56B150EC46FE9DC3E
:1048200002C0C2F001C0C1F0BE510124016E000EF1
:104830000220036E015003C0F7FF59EC09F0016E2E
:10484000C05D1EE002EC19F0460EF66E290EF76E02
:10485000196AF2BE198EF29E3A0E0101266F00010E
:1048600030EC1AF019BEF28E070E04009EA8FDD798
:10487000AD6E200E04009EA8FDD7AD6E9C953ED275
:10488000BE2B99D7BF2BBF51340801E2BF6BAA6A78
:10489000340EA96EBFC0A8FFA69CA69EA684F250A7
:1048A000006EF29E0F01550EA76EAA0EA76EA6828D
:1048B000A6B2FED7A6940050F2120001C2D1F2CFE8
:1048C000C1F0F29EAA6A350EA96EA69CA69EA6808D
:1048D000A850C1BFF28EBF6FBE6BBE51140865E316
:1048E00082DC036ABE5157EC00F0C16FC36BBFC0DE
:1048F000C2F0C56B150EC46F7CDC02C0C3F001C0F2
:10490000C2F0BE510124016E000E0220036E015060
:1049100003C0F7FF8DEC0BF0C26FC1C0C3F0C46FD2
:1049200058EC20F009DC036ABE5157EC00F0C16F6F
:10493000C26FA1DC01C0C0F0C36BBFC0C2F0C56BC9
:10494000150EC46F56DC02C0C2F001C0C1F0BE51EA
:104950000124016E000E0220036E015003C0F7FF18
:104960008DEC0BF0016EC05D1EE002EC19F0460EFE
:10497000F66E290EF76E196AF2BE198EF29E3A0E85
:104980000101266F000130EC1AF019BEF28E070EFD
:1049900004009EA8FDD7AD6E200E04009EA8FDD792
:1049A000AD6E9C95ABD1BE2B98D7BF2BBF513508B0
:1049B00001E2BF6BAA6A350EA96EBFC0A8FFA69C14
:1049C000A69EA684F250006EF29E0F01550EA76EB1
:1049D000AA0EA76EA682A6B2FED7A6940050F21227
:1049E00000012FD1F2CFC1F0F29EAA6A360EA96E55
:1049F000A69CA69EA680A850C1BFF28EBF6FBE6BBC
:104A0000BE51140869E3F3EC20F0036ABE5157EC81
:104A100000F0C16FC36BBFC0C2F0C56B150EC46F91
:104A2000F9EC20F002C0C3F001C0C2F0BE51012475
:104A3000016E000E0220036E015003C0F7FFCBECA5
:104A40000DF0C26FC1C0C3F0C46F58EC20F09CECF5
:104A500020F0036ABE5157EC00F0C16FC26F0BDC4F
:104A600001C0C0F0C36BBFC0C2F0C56B150EC46FF0
:104A7000F9EC20F002C0C2F001C0C1F0BE51012427
:104A8000016E000E0220036E015003C0F7FFCBEC55
:104A90000DF0016EC05D1EE002EC19F0460EF66EE0
:104AA000290EF76E196AF2BE198EF29E3A0E0101B6
:104AB000266F000130EC1AF019BEF28E070E0400CA
:104AC0009EA8FDD7AD6E200E04009EA8FDD7AD6E4A
:104AD0009C9514D1BE2B94D7BF2BBF51350801E252
:104AE000BF6BAA6A360EA96EBFC0A8FFA69CA69E81
:104AF000A684F250006EF29E0F01550EA76EAA0E0C
:104B0000A76EA682A6B2FED7A6940050F2120001AC
:104B100098D0F2CFC1F0F29EAA6A370EA96EA69C79
:104B2000A69EA680A850C1BFF28EBF6FBE6BBE51BD
:104B300014086AE3F3EC20F0036ABE5157EC00F06E
:104B4000C16FC36BBFC0C2F0C56B150EC46FF9EC6B
:104B500020F002C0C3F001C0C2F0BE510124016EBA
:104B6000000E0220036E015003C0F7FF09EC10F0A5
:104B7000C26FC1C0C3F0C46F58EC20F09CEC20F0B1
:104B8000036ABE5157EC00F0C16FC26F3BEC21F0DD
:104B900001C0C0F0C36BBFC0C2F0C56B150EC46FBF
:104BA000F9EC20F002C0C2F001C0C1F0BE510124F6
:104BB000016E000E0220036E015003C0F7FF09ECE6
:104BC00010F0016EC05D1EE002EC19F0460EF66EAC
:104BD000290EF76E196AF2BE198EF29E3A0E010185
:104BE000266F000130EC1AF019BEF28E070E040099
:104BF0009EA8FDD7AD6E200E04009EA8FDD7AD6E19
:104C00009C957CD0BE2B93D7BF2BBF51340801E2BB
:104C1000BF6BAA6A370EA96EBFC0A8FFA69CA69E4E
:104C2000A684F250006EF29E0F01550EA76EAA0EDA
:104C3000A76EA682A6B2FED7A6940050F21200017B
:104C400000D0C06BBE6BBE51790808E3BEC0C2F095
:104C50003BEC21F00150C01BBE2BF5D7F3EC20F04C
:104C60007A0EC36FC0C0C4F058EC20F09CEC20F06A
:104C70007A0EC26F3BEC21F00150C05D10E002ECF7
:104C800019F06C0EF66E3C0EF76E196AF2BE198EB4
:104C9000F29E9EEC19F019BEF28E9C952FD0F3EC8B
:104CA00020F07D0EC36FC0C0C4F058EC20F09CEC27
:104CB00020F07D0EC26F3BEC21F00150C05D10E092
:104CC00002EC19F0AE0EF66E3C0EF76E196AF2BEEB
:104CD000198EF29E9EEC19F019BEF28E9C950ED0A4
:104CE000F00EF66E3C0EF76E196AF2BE198EF29E49
:104CF0009EEC19F019BEF28E02EC00F072EF27F074
:104D0000E824F76AF7361B0FF66E4D0EF7220A00FD
:104D1000F550FA6E0800F550F96E04432C445245E4
:104D200076469A47BE48E449124BEACFE0F0E9CF15
:104D3000DFF0D939F009DB6FDB27E20FDC6F320FD0
:104D4000DE6FD9510F0BDC27DC27DE27E90FDD6F83
:104D5000DD27DD27D8390F0BDD27DE27DD37DE37EE
:104D6000DE1FDE37D8510F0BDE27DB37070EDA6F79
:104D70000A0EDD07DE27FDE3DC07DD27FDE3DB07A9
:104D8000DC27FDE3DA07DB27FDE3EA6ADA0EE96EEA
:104D9000070EDF15DF9DE926DE0EE95CD8B4DF8D56
:104DA000EF50006E08E1DFBD06D0DFB90DD0DFB7F0
:104DB00002D0200E03D0DF87DF99300E002600508E
:104DC00004009EA8FDD7AD6EEE50DFADE5D7000C18
:104DD000BE6BBD6B02EC19F0F2CFBFF0F29EAA6A77
:104DE000100EA96EA69CA69EA680A850BFBFF28EEC
:104DF000C06FF2CFC1F0F29EAA6A110EA96EA69CF6
:104E0000A69EA680A850C1BFF28EC26FC0C0BEF0E1
:104E1000C2C0BDF0010EBD5F000EBE5BBEC0BFF0E4
:104E2000C06BAA6A100EA96EBFC0A8FFA69CA69E62
:104E3000A684F250006EF29E0F01550EA76EAA0EC8
:104E4000A76EA682A6B2FED7A6940050F212AA6A56
:104E5000110EA96EBDC0A8FFA69CA69EA684F2CF87
:104E600000F0F29E550EA76EAA0EA76EA682A6B2FD
:104E7000FED7A6940050F212400EF66E3D0EF76E6D
:104E8000196AF2BE198EF29E00019EEC19F019BE4D
:104E9000F28E660EF66E3D0EF76E196AF2BE198E30
:104EA000F29E210E0101266F000130EC1AF019BEAE
:104EB000F28E100EE96EBEC0D9F0BDC0D8F035DF5D
:104EC0000A0E04009EA8FDD7AD6E0D0E04009EA82C
:104ED000FDD7AD6E75EF27F0BB5304E0BCC0BDF04D
:104EE00078EF21F09CA501D073D7080EBD6FFA0EA4
:104EF000D16F06EC20F0BD2FFAD7196AF2BE198ED9
:104F0000F29E80EC1DF019BEF28EF294F28A000C33
:104F100002EC19F0820EF66E3E0EF76E196AF2BEC2
:104F2000198EF29E9EEC19F019BEF28E080EBB6F20
:104F3000FA0ED16F06EC20F0BB2FFAD7196AF2BE39
:104F4000198EF29E80EC1DF019BEF28EF294F28A58
:104F5000000CBF51BE5D4AE07A0EC36FBEC0C4F004
:104F600058EC20F09CEC20F0520EF66E2E0EF76EF0
:104F7000196AF2BE198EF29E220E0101266F0001FF
:104F800030EC1AF019BEF28E196AF2BE198EF29E3A
:104F9000BFC026F1370E0101276F000146EC1AF061
:104FA00019BEF28E770EF66E2E0EF76E196AF2BEED
:104FB000198EF29E070E0101266F000130EC1AF0E7
:104FC00019BEF28E196AF2BE198EF29EBEC026F18B
:104FD000370E0101276F000146EC1AF019BEF28E60
:104FE0000A0E04009EA8FDD7AD6E0CD0840EF66E9E
:104FF0002E0EF76E196AF2BE198EF29E9EEC19F013
:1050000019BEF28E54EF2EF0D8B203D0EA6AD90E50
:10501000E96E006A016A026A036AD96BDA6BDB6BBC
:10502000DC6BD851D711D611D5112CE0200EDD6FD5
:10503000D890D137D237D337D437D937DA37DB37AF
:10504000DC37D851DC5D08E1D751DB5D05E1D65195
:10505000DA5D02E1D551D95D0FE3D551D95FD65163
:10506000D8A0D63DDA5FD751D8A0D73DDB5FD85165
:10507000D8A0D83DDC5FD880003601360236033632
:10508000DD2FD6D7D9C0EFFFDAC0ECFFDBC0ECFFD5
:10509000DCC0ECFF000CE950C96F3B0ED06F9A0EDC
:1050A000CF6FCA0ECE6FCD6B0A0ECB6FD882EA6A75
:1050B000C50EE96EC8C0D4F0C7C0D3F0C6C0D2F0E8
:1050C000C5C0D1F0D0C0D8F0CFC0D7F0CEC0D6F098
:1050D000CDC0D5F099DF015000520FE1CB51010A4C
:1050E0000CE0C9510BE00F0BCB5D01E00EE2C9BF34
:1050F0000CD0C9BD03D0200E02D0C96B300E0026E3
:10510000005004009EA8FDD7AD6ED892D0C0D4F058
:10511000CFC0D3F0CEC0D2F0CDC0D1F0D86BD76B1A
:10512000D66B0A0ED56F70DF03C0D0F002C0CFF08F
:1051300001C0CEF000C0CDF0CB2FB8D7DCEF28F007
:10514000C26B40C0C1F041C0C0F042C0BFF0C2332A
:10515000C133C033BF33C233C133C033BF333F0E5B
:10516000C217BE530CE07E0EF66E2A0EF76E196A59
:10517000F2BE198EF29E9EEC19F019BEF28E196ADB
:10518000F2BE198EF29E010E0101266F250E276FC9
:10519000280E286F00016FEC19F019BEF28EBE5375
:1051A00010E0410EE96EC2C0C8F0C1C0C7F0C0C077
:1051B000C6F0BFC0C5F06FD72D0E04009EA8FDD766
:1051C000AD6E35C0C2F036C0C1F037C0C0F038C0D7
:1051D000BFF0C233C133C033BF33C233C133C03376
:1051E000BF33C233C133C033BF33C233C133C03323
:1051F000BF33C233C133C033BF33C233C133C03313
:10520000BF33C233C133C033BF33010EC217BF51E6
:105210001F0BC46FC233C133C033BF33C233C1337A
:10522000C033BF33C233C133C033BF33C233C133E2
:10523000C033BF33C233C133C033BF33070EC217CD
:10524000BF513F0BC36FBE5330E0196AF2BE198ED7
:10525000F29EC3C029F11B0E01012A6F00012DEC43
:1052600019F019BEF28E2D0E04009EA8FDD7AD6E6A
:10527000196AF2BE198EF29EC4C029F11B0E0101FB
:105280002A6F00012DEC19F019BEF28E200E0400D9
:105290009EA8FDD7AD6E200E04009EA8FDD7AD6E72
:1052A000200E04009EA8FDD7AD6E196AF2BE198EBD
:1052B000F29EB0EC19F019BEF28E6AEF2EF0C06BC0
:1052C000BF6BBE530CE0960EF66E2A0EF76E196A8F
:1052D000F2BE198EF29E9EEC19F019BEF28EC06BD2
:1052E00044C0BFF04550BF27000EC0234650BF2723
:1052F000000EC0234750BF27000EC0234850BF27D1
:10530000000EC0234D50BF27000EC0234E50BF27B4
:10531000000EC0234F50BF27000EC0235050BF27A0
:10532000000EC023196AF2BE198EF29E010E010111
:10533000266F250E276F280E286F00016FEC19F0DD
:1053400019BEF28EBFC000F0C0C003F0030EC05DF6
:1053500003E1F70E005C07E0040E035C03E1610E5D
:10536000005C14E026D0BE530CE0840EF66E290ECD
:10537000F76E196AF2BE198EF29E9EEC19F019BEF4
:10538000F28E030EC26F070EC16F22D0BE530CE027
:105390008E0EF66E290EF76E196AF2BE198EF29E07
:1053A0009EEC19F019BEF28E010EC26F900EC16F05
:1053B0000FD0BE530CE0980EF66E290EF76E196AE8
:1053C000F2BE198EF29E9EEC19F019BEF28E00D03C
:1053D000196AF2BE198EF29EB0EC19F019BEF28E67
:1053E000C1C001F0C2C002F06EEF2EF08E0E006E52
:1053F000D4C001F0D3C002F0036A015209E102C037
:1054000001F0026A080E005E015202E1006A08D053
:10541000D89001BE04D0023601360006F9D7019EAD
:10542000000CD151D8B4A5D0DD6FD551D8B4A1D0DE
:10543000DD5F05E37F0EDD27D8B09BD006D0810E5F
:10544000DD5FD8A096D0D8B494D0DDC000F0016A5A
:10545000026A036ADC6BD2C0DBF0DB8FD3C0DAF008
:10546000D4C0D9F0190EDD6FD851D95F0DE2010E0D
:10547000DA5F0AE2DB5F08E2DC5F06E2DC2BDB2BB3
:10548000DA2BD851D92728D0D751DA5F12E2010E92
:10549000DB5F0FE2DC5F0DE2DC2BDB2BD751DA2781
:1054A000D851D92719E3DA2B17E1DB2B15E1DC2BD7
:1054B00013D0D6518009DB5F0EE2010EDC5F0BE2F8
:1054C000DC2BD6518009DB27D751DA27E9E3DB2B28
:1054D000E7E1DC2BE5D70380DD2F01D00BD0D8909E
:1054E000D937DA37DB37DC37D89003360236013666
:1054F000DE37BAD7DEA106D0D890013202320332AD
:10550000DE3302D0000635E0DEBF1ED0D890D9379A
:10551000DA37DB37DC37D851D95F07E2010EDA5FC3
:1055200004E2DB5F02E2DC5F1AE3D751DA5F05E2F7
:10553000010EDB5F02E2DC5F12E3D6518009DB5F24
:1055400003E2010EDC5F0BE3032A09E1022A07E113
:10555000012A05E1002A0DE0013202320332D2C0F5
:10556000DDF0D651DD1BDDAF02D0018E06D0019EED
:1055700004D0006A016A026A036AB7EF2CF0D351C3
:10558000D8B471D0006ED751D8B46DD0002604E3E2
:10559000810E002668E204D07F0E005E64E363E0C3
:1055A000D4C0DBF0D851DB1BD48FD88FD651DA03AF
:1055B000F4CFDDF0D551D903F4CF03F0F3CFDCF015
:1055C000DA03F350DD27F450DC23000E0322D6511A
:1055D000D903F350DD27F450DC23000E026A0322C6
:1055E0000222D451DA03F350DC27F4500322000ED8
:1055F0000222D451D903F3500326F4500222000EA4
:10560000016A0122D651D803F350DC27F45003225B
:10561000000E02220122D551D803F3500326F45084
:105620000222000E0122D451D803F3500226F45076
:105630000122002A01BE05D0DC37033602360136CE
:105640000006000EDCAF0AD0032A0222012201501C
:1056500005E1025003E1035001E1002ADBBF018EA6
:10566000DBAF019E04D0006A016A026A036AFAEFA6
:105670002CF0800ED8B2D61BDB6BDC6BD2C0DAF01C
:10568000D651DA1BD151D8B4DCD0D96F006ED551C8
:10569000D8B4E0D0D95FD8B481D03DE3D6C0DFF034
:1056A000DF8FD7C0DEF0D8C0DDF0DC6BD890DF3301
:1056B000DE33DD33DC33D92FF8D7DAAF03D0DB812B
:1056C000DDD0DB91D991DB89EA6AD40EE96EE9D0AD
:1056D000DB99DABF0AD0D9A113D0DF33DE33DD3353
:1056E000DC33002AD8B4C5D00BD0DFBF0CD0D890A3
:1056F000DC37DD37DE37DF370006D8B4BAD0F5D770
:10570000DB8D6BD0DB9DD2C0DAF0D2AF02D0DF8F61
:10571000A9D0DF9FA7D0D5C0D9F0D5C000F0D15116
:10572000D95FD2C0DFF0DF8FD3C0DEF0D4C0DDF0B0
:10573000DC6BD890DF33DE33DD33DC33D92FF8D7A1
:10574000DAAF03D0DB839AD0DB93D991DB8BEA6AA3
:10575000D80EE96EA6D0DB9BDABF0AD0D9A113D050
:10576000DF33DE33DD33DC33002AD8B482D00BD014
:10577000DFBF0CD0D890DC37DD37DE37DF370006EF
:10578000D8B477D0F5D7DB8F28D0DB9FD6C0DAF03E
:10579000D6AF02D0DF8F66D0DF9F64D0D6C0DFF0F7
:1057A000DF8FD7C0DEF0D8C0DDF0DAAF04D0DF9FE6
:1057B000DB8564D0DB95DC6BD991EA6AD40EE96EA7
:1057C00070D0DABF1CD0D2C0DAF0D9A106D0DF3356
:1057D000DE33DD33DC33002A4CE0DCAF0BD0DD2BD5
:1057E00009E1DE2B07E1DF2B05E1DF33DE33DD33BB
:1057F000002A3FE0DBBD86D7DBBFC7D71CD0800EB9
:10580000DF1BDFAF04D03AD0D6C0DAF00AD0D2C066
:10581000DAF0DF5306E1DE5304E1DD5302E1006A12
:1058200021D0DFBF08D0D890DC37DD37DE37DF3757
:10583000002EF7D71ED0DAAF02D0DF8F13D0DF9F54
:1058400011D0D5C000F0D6C0DFF0D7C0DEF0D8C090
:10585000DDF008D0D1C000F0D2C0DFF0D3C0DEF060
:10586000D4C0DDF0DFC001F0DEC002F0DDC003F027
:1058700034D0006A016A026A036A2FD0DC6BDD1F34
:10588000DE1FDF1FDC1FDC2B05E1DD2B03E1DE2B40
:1058900001E1DF2BDBB115D7DBB356D7DBB58AD7F8
:1058A000B3D7EF50DD2705E3DE2B03E1DF2BD8B4C0
:1058B000D981ED52EF50DE2703E3DF2BD8B4D98135
:1058C000ED52EF50EFBE01D0800ADF27D8B0D9816A
:1058D000DBB9FED6DBBB3FD774D716EF2DF08E0EAB
:1058E000006ED151005ED2C002F0D3C001F0028E32
:1058F000005209E0D890025202E1015204E0023263
:105900000132002EF7D7D2AF05D0011E021E012AA8
:10591000D8B4022A000CC191D06BCF6BCE6BCD6B8B
:10592000BF31036EBE31026E0332023203320232E5
:105930001F0E031602C0D3F003C0D4F057DD03C01E
:10594000C8F002C0C7F001C0C6F000C0C5F0C8C0B2
:10595000D4F0C7C0D3F0C6C0D2F0C5C0D1F0D86B68
:10596000FF0ED76F7F0ED66F8E0ED56F5AD503C040
:10597000CCF002C0CBF001C0CAF000C0C9F029527F
:105980000EE1BFC0D4F0BEC0D3F030DD03C0D0F014
:1059900002C0CFF001C0CEF000C0CDF051D0C26B3C
:1059A000C25107084DE329C000F0C251016E04E066
:1059B000D8900032012EFCD700B040D0C1B124D025
:1059C00080C0D2F081C0D1F080C0D4F081C0D3F0CB
:1059D0000DDD03C0D6F002C0D5F001C0D4F000C088
:1059E000D3F0CCC0DAF0CBC0D9F0CAC0D8F0C9C06F
:1059F000D7F0C5D503C0D0F002C0CFF001C0CEF0C3
:105A000000C0CDF0C1811AD0D892D0C0D4F0CFC0A0
:105A1000D3F0CEC0D2F0CDC0D1F0C8C0D8F0C7C04E
:105A2000D7F0C6C0D6F0C5C0D5F023D603C0D0F09D
:105A300002C0CFF001C0CEF000C0CDF0C22BB0D775
:105A4000D0C0D4F0CFC0D3F0CEC0D2F0CDC0D1F012
:105A500046DF02C0C4F001C0C3F0C0533CE0A20E58
:105A6000F66E2A0EF76E196AF2BE198EF29E9EEC41
:105A700019F019BEF28E196AF2BE198EF29E010E4D
:105A80000101266F250E276F280E286F00016FEC8D
:105A900019F019BEF28E100EE96EC4C0D9F0C3C061
:105AA000D8F095EC26F0B10EF66E2A0EF76E196A54
:105AB000F2BE198EF29E050E0101266F000130EC38
:105AC0001AF019BEF28E196AF2BE198EF29EB0EC6F
:105AD00019F019BEF28ED0C0D4F0CFC0D3F0CEC032
:105AE000D2F0CDC0D1F0FBDE025079EF2EF0BB6BCF
:105AF000B95326E002EC19F0196AF2BE198EF29E33
:105B0000010E0101266F250E276F280E286F000158
:105B10006FEC19F019BEF28E780EF66E3B0EF76E32
:105B2000196AF2BE198EF29E9EEC19F019BEF28E21
:105B3000196AF2BE198EF29EB0EC19F019BEF28EFF
:105B4000B853D8A4D7D0BA6BBA517F0816E3036A0A
:105B5000BA511C0F016E000E032201C0BEF003C03B
:105B6000BFF0BAC0C2F03BEC21F0BFC0EAFFBEC03C
:105B7000E9FF01C0EFFFBA2BE7D7B953D8B47DD006
:105B8000BA6BBA517F08D8A078D0BA510F0B57E141
:105B9000196AF2BE198EF29E010E0101266F250EC2
:105BA000276F280E286F00016FEC19F019BEF28ED6
:105BB0000D0E04009EA8FDD7AD6E0A0E04009EA82F
:105BC000FDD7AD6E196AF2BE198EF29EBAC026F1EB
:105BD000370E0101276F000146EC1AF019BEF28E54
:105BE0003A0E04009EA8FDD7AD6E196AF2BE198E5A
:105BF000F29EB0EC19F019BEF28E036ABA511C0F76
:105C0000E96E000E0320EA6EEFCFBEF0200E040016
:105C10009EA8FDD7AD6E196AF2BE198EF29EBEC067
:105C200026F1370E0101276F000146EC1AF019BE6C
:105C3000F28E200E04009EA8FDD7AD6E1CD0036A24
:105C4000BA511C0FE96E000E0320EA6EEFCFBEF0D2
:105C5000196AF2BE198EF29EBEC026F1370E0101FE
:105C6000276F000146EC1AF019BEF28E200E0400D8
:105C70009EA8FDD7AD6EBA2B84D7BA6BBA517908FE
:105C80000BE3036ABA511C0FE96E000E0320EA6EA3
:105C9000EF50BB1BBA2BF2D7B95306E0BBC0BEF026
:105CA00096C0BFF0A9EF27F0B95323E03F50680832
:105CB0000DE0B00EF66E3B0EF76E196AF2BE198E4D
:105CC000F29E9EEC19F019BEF28E13D0B9C0BEF050
:105CD000A0EF28F0B9C0BEF05FEF29F002C0BDF020
:105CE00001C0BCF0BDC0BFF0BCC0BEF0B9C0C0F0C8
:105CF00012D681D1BA6BBA517F08D8A07CD1800E60
:105D0000BA25BE6FF2CFBFF0F29EAA6ABEC0A9FF4D
:105D1000A69CA69EA680A850BFBFF28EBE6F196A31
:105D2000F2BE198EF29EBEC026F1370E0101276F1A
:105D3000000146EC1AF019BEF28E200E04009EA857
:105D4000FDD7AD6EBA51780810E3800EBA25BE6F4C
:105D5000F2CFBFF0F29EAA6ABEC0A9FFA69CA69E83
:105D6000A680A850BFBFF28EBB1BBA517F08D8A433
:105D700040D1FA0EF66E3B0EF76E196AF2BE198E1E
:105D8000F29E9EEC19F019BEF28EF2CFBEF0F29E9A
:105D9000AA6A800EA96EA69CA69EA680A850BEBF29
:105DA000F28E000A29E0010A35E0030A41E0010A07
:105DB0004DE0070A59E0010A65E0030AD8B470D043
:105DC000010AD8B47BD00F0AD8B486D0010AD8B45F
:105DD00091D0030AD8B49CD0010AD8B4A7D0070A3E
:105DE000D8B4B2D0010AD8B4BDD0030AD8B4C8D050
:105DF000010AD8B4D3D0E0D09C81920EF66E280E62
:105E0000F76E196AF2BE198EF29E9EEC19F019BE59
:105E1000F28EE0D09C81EC0EF66E280EF76E196AB9
:105E2000F2BE198EF29E9EEC19F019BEF28ED2D0FF
:105E30009C81740EF66E280EF76E196AF2BE198EEA
:105E4000F29E9EEC19F019BEF28EC4D09C810A0E0F
:105E5000F66E290EF76E196AF2BE198EF29E9EEC4E
:105E600019F019BEF28EB6D09C81B00EF66E280ED7
:105E7000F76E196AF2BE198EF29E9EEC19F019BEE9
:105E8000F28EA8D09C81280EF66E290EF76E196A44
:105E9000F2BE198EF29E9EEC19F019BEF28E9AD0C7
:105EA0009C81560EF66E280EF76E196AF2BE198E98
:105EB000F29E9EEC19F019BEF28E8CD09C81CE0E13
:105EC000F66E280EF76E196AF2BE198EF29E9EECDF
:105ED00019F019BEF28E7ED09C81920EF66E280EBD
:105EE000F76E196AF2BE198EF29E9EEC19F019BE79
:105EF000F28E70D09C81EC0EF66E280EF76E196A49
:105F0000F2BE198EF29E9EEC19F019BEF28E62D08E
:105F10009C81740EF66E280EF76E196AF2BE198E09
:105F2000F29E9EEC19F019BEF28E54D09C810A0E9E
:105F3000F66E290EF76E196AF2BE198EF29E9EEC6D
:105F400019F019BEF28E46D09C81B00EF66E280E66
:105F5000F76E196AF2BE198EF29E9EEC19F019BE08
:105F6000F28E38D09C81280EF66E290EF76E196AD3
:105F7000F2BE198EF29E9EEC19F019BEF28E2AD056
:105F80009C81560EF66E280EF76E196AF2BE198EB7
:105F9000F29E9EEC19F019BEF28E1CD09C81CE0EA2
:105FA000F66E280EF76E196AF2BE198EF29E9EECFE
:105FB00019F019BEF28E0ED09C911C0EF66E3C0E9E
:105FC000F76E196AF2BE198EF29E9EEC19F019BE98
:105FD000F28E00D00D0E04009EA8FDD7AD6E0A0E05
:105FE00004009EA8FDD7AD6E0A0E04009EA8FDD742
:105FF000AD6EBA2B80D6000CB20EF66E2B0EF76E7D
:10600000196AF2BE198EF29E9EEC19F019BEF28E3C
:10601000D19004009EAAFDD7AE50D180000C0400A0
:106020009EA8FDD7AD6E000C04009EAAFDD7AECF92
:10603000D5F0D551F4DFD551390805E3300ED55DE3
:10604000016E0FD00ED0D551600806E2D5517A0806
:1060500003E3D551DF0B01D0D551BF0F0A0F016EFD
:1060600000D0000CE1DF01C0D4F0DEDF01C0D3F0CE
:10607000D351DD0804E1D4C001F007D006D0D451DB
:10608000100DF350D325016E00D0000C620EF66E99
:106090002B0EF76E196AF2BE198EF29E9EEC19F065
:1060A00019BEF28EDFDF01C0BBF0BBC001F005EF0F
:1060B00031F0200EBEA9300EBF6FBDC000F0BDAFE5
:1060C00007D0001E002A00C0BDF02D0EBF6FBE8F8E
:1060D0000150196AF2BE198EF29EBDC02BF1640EFA
:1060E00001012C6F000117EC19F019BEF28E00C0EF
:1060F000BDF0300E0124C06F196AF2BE198EF29EF7
:10610000BDC02BF10A0E01012C6F000117EC19F034
:1061100019BEF28E300E0024C26F300E0124C16F02
:10612000BFC000F0BEA702D0BEAFBE95BEB90BD0B7
:10613000BEAF22D0BEB520D000C0C0F0BEB31CD0D0
:1061400000C0C1F019D0300EC05D16E100C0C0F033
:10615000200EBF6FBEA704D0BE95BE83BEAFBE9358
:10616000300EC15D09E100C0C1F0200EC06FBEA7B6
:10617000F7D7BE93BEAFBE91BEA505D0BF510400F8
:106180009EA8FDD7AD6EBEA305D0C05104009EA849
:10619000FDD7AD6EBEA105D0C15104009EA8FDD7AC
:1061A000AD6EC25104009EA8FDD7AD6EEDEF30F08C
:1061B0008A0EF66E2B0EF76E196AF2BE198EF29EDB
:1061C000140E0101266F000130EC1AF019BEF28E98
:1061D000BBC0BDF01F0EBE6F6CD7A00EF66E2B0EAF
:1061E000F76E196AF2BE198EF29E100E0101266F2B
:1061F000000130EC1AF019BEF28E34DF01C0BCF0A1
:10620000BCC001F00AEF31F041D701C0B8F0010E77
:10621000BB6FCED701C0BAF003EC20F0B8518008B4
:1062200002E2F3EC20F0B8C0C3F0BAC0C4F058ECFE
:1062300020F002EC00F0B851800802E2F3EC20F00C
:10624000B8C0C2F03BEC21F001C0B9F0BA51B95D61
:106250000DE12C0EF66E3C0EF76E196AF2BE198E29
:10626000F29E9EEC19F019BEF28E3CD0400EF66EF6
:106270003C0EF76E196AF2BE198EF29E1E0E0101D7
:10628000266F000130EC1AF019BEF28E196AF2BEC8
:10629000198EF29EBAC026F1370E0101276F000158
:1062A00046EC1AF019BEF28E610EF66E3C0EF76ED9
:1062B000196AF2BE198EF29E060E0101266F0001C8
:1062C00030EC1AF019BEF28E196AF2BE198EF29EE7
:1062D000B9C026F1370E0101276F000146EC1AF014
:1062E00019BEF28E89DE16EF41F0BB6BBA6BF2CFAE
:1062F000BCF0F29EAA6A100EA96EA69CA69EA6806D
:10630000A850BCBFF28EBD6FF2CFBEF0F29EAA6A5B
:10631000110EA96EA69CA69EA680A850BEBFF28EA6
:10632000BF6FBDC0BBF0BFC0BAF0BAC001F0BBC008
:1063300002F09CEF31F0D9D702C0B9F001C0B8F03B
:106340001C0EF66E3D0EF76E196AF2BE198EF29EA5
:106350001D0E0101266F000130EC1AF019BEF28EFD
:10636000100EE96EB9C0D9F0B8C0D8F095EC26F09F
:106370000A0E04009EA8FDD7AD6E0D0E04009EA867
:10638000FDD7AD6E3BEF41F0DB07DC6B04009EAA4E
:10639000FDD7AECFDDF0DD5108080AE1DC5307E0A0
:1063A000DC07DD513CDE200E3ADEDD5138DE15D053
:1063B000DD511F0812E2DD517E080FE3DC51DB5D89
:1063C0000CE3DC51DC2B036AD925E96EDA5103209A
:1063D000EA6EDDC0EFFFDD5122DEDD510D08D6E1B2
:1063E000036ADC51D925E96EDA510320EA6EEF6ABF
:1063F000000CE251E419800BE66FE2AF05D0E11F1B
:10640000E21FE12BD8B4E22BE4AF05D0E31FE41F79
:10641000E32BD8B4E42BE151E303F3CF01F0F4CF45
:1064200000F0E403F3500026E251E303F3500020B0
:10643000026EE6AF05D0011E021E012AD8B4022A60
:1064400093EF32F0DF6BDD6B0A0EDE6FDC6BDB6B24
:10645000D951DA1104E1000E016E026EE6D0DF516F
:10646000DF2B036AD925E96EDA510320EA6EEFCFFC
:10647000E0F0E0512D080DE1010EDD6FDF51DF2B63
:10648000036AD925E96EDA510320EA6EEFCFE0F016
:106490000DD0E0512B080AE1DF51DF2B036AD9252B
:1064A000E96EDA510320EA6EEFCFE0F0E0512F08F9
:1064B000D8B0ADD0E0513908D8A0A9D0E05130080B
:1064C00021E1036ADF51D925E96EDA510320EA6E32
:1064D000EF5078080AE0036ADF51D925E96EDA51F6
:1064E0000320EA6EEF5058080DE1100EDE6FDF2B2F
:1064F000DF51DF2B036AD925E96EDA510320EA6EFA
:10650000EFCFE0F0DE510A0821E1E0512F081DE253
:10651000E05139081AE3E26B0A0EE16FDCC0E4F0E7
:10652000DBC0E3F066D7300EE05D0124DB6F000EC8
:106530000220DC6FDF51DF2B036AD925E96EDA51C7
:106540000320EA6EEFCFE0F0E0D761D0DE51100813
:106550005EE1E051600806E2E0517A0803E3E051B1
:10656000DF0B01D0E051E06FE0512F0803E2E05172
:10657000390806E2E05140084AE2E051460847E3A4
:10658000E0512F0819E2E051390816E3DB35E16FDD
:10659000DC35E26FE137E237E137E237E137E23706
:1065A000F00EE117300EE05DE125016E000EE221F4
:1065B00001C0DBF0DC6F16D0DB35E16FDC35E26F5C
:1065C000E137E237E137E237E137E237F00EE11742
:1065D000410EE05D0A0FE125016E000EE22101C0CF
:1065E000DBF0DC6FDF51DF2B036AD925E96EDA516E
:1065F0000320EA6EEF50E06F600806E2E0517A088F
:1066000003E3E051DF0B01D0E051E06FADD7DE5185
:106610000A0807E1DD2D05D0DB1FDC1FDB2BD8B41A
:10662000DC2BDBC001F0DCC002F021EF33F0DA6BD1
:10663000D00ED96F070EDB6FA7DEDA6BD00ED96FE5
:1066400001D702C0D8F001C0D7F0D7C001F0D8C040
:1066500002F0000C010E0101236F2351225D07E3BC
:106660001E31213320331F331E33232BF6D71EC197
:1066700000F01FC101F020C102F021C103F00001B0
:10668000000C010E0101236F2351225D07E3213528
:106690001E371F3720372137232BF6D71EC100F0B6
:1066A0001FC101F020C102F021C103F00001000C64
:1066B000120EDB6F340EDA6F560ED96F780ED86F6C
:1066C000010ED66FD6510A083AE3D651040DF350A5
:1066D000036AD80F016E000E032201C018F103C037
:1066E00019F1010E0001D65D040DF350036AD80FB5
:1066F000E96E000E0320EA6EEFCF1AF1ECCF1BF12A
:10670000ECCF1CF1ECCF1DF11DC121F11CC120F11A
:106710001BC11FF11AC11EF1020E0101226F0001FF
:1067200099DF19C1EAFF18C1E9FF00C0EFFF01C0FE
:10673000ECFF02C0ECFF03C0ECFFD62BC3D7F2CFB7
:1067400018F1F29EAA6A200EA96EA69CA69EA680AB
:10675000A850010118BFF28E196FF2CF1AF1F29E04
:10676000AA6A210EA96EA69CA69EA680A8501ABF52
:10677000F28E1B6FD0C006F1D1C007F119C105F12F
:106780001BC104F19A0E0B6FBC0E0A6FDE0E096F6F
:10679000F00E086FF2CF18F1F29EAA6A220EA96ECF
:1067A000A69CA69EA680A85018BFF28E196F19C18C
:1067B0000FF1FF0E0E6FFF0E0D6F800E0C6F136B3F
:1067C000126B116B106B176B166B010E156FB80EF9
:1067D000146F670E0001A66F450EA56F230EA46F00
:1067E000010EA36FEF0EAA6FCD0EA96FAB0EA86FAF
:1067F000890EA76F980EAE6FBA0EAD6FDC0EAC6F40
:10680000FE0EAB6F100EB26F320EB16F540EB06F42
:10681000760EAF6FC30EB66FD20EB56FE10EB46FCA
:10682000F00EB36FD66BD6514F08D8A04CD3D651CB
:106830000F0BD76FD6510F08D8B08CD0D751040D9D
:10684000F350036AD80F016E000E032201C018F145
:1068500003C019F10D0E0001D7250F0B040DF350E5
:10686000036AD80FE96E000E0320EA6EEFCF1AF12B
:10687000ECCF1BF1ECCF1CF1ECCF1DF1080ED725AE
:106880000F0B040DF350036AD80FE96E000E0320BE
:10689000EA6EEFCF00F0ECCF01F0ECCF02F0ECCFDE
:1068A00003F0005001011A1B01501B1B02501C1B5E
:1068B00003501D1B020E0001D7250F0B040DF350D2
:1068C000036AD80FE96E000E0320EA6EEFCF00F0E6
:1068D000ECCF01F0ECCF02F0ECCF03F0005001015F
:1068E0001A1B01501B1B02501C1B03501D1B0001D7
:1068F000D751040DF350036AD80FE96E000E032040
:10690000EA6EEFCF00F0ECCF01F0ECCF02F0ECCF6D
:1069100003F0005001011A1B01501B1B02501C1BED
:1069200003501D1B1DC121F11CC120F11BC11FF112
:106930001AC11EF1010E226F0001A3DE19C1EAFF88
:1069400018C1E9FF00C0EFFF01C0ECFF02C0ECFF7F
:1069500003C0ECFFD651130802E2000E01D0010E75
:10696000010BD8B49ED0A6C021F1A5C020F1A4C0CF
:106970001FF1A3C01EF1050E0101226F000181DE8F
:1069800003C01BF102C01AF101C019F100C018F1D7
:10699000A751AB1501011C6F0001A851AC150101F5
:1069A0001D6F0001A951AD1501011E6F0001AA5113
:1069B000AE1501011F6FA7C020F10101201FA8C063
:1069C00021F10101211FA9C022F10101221FAAC04A
:1069D00023F10101231F20510001AF15006E0101B9
:1069E00021510001B015016E010122510001B115C4
:1069F000026E010123510001B215036E0050010126
:106A00001C11006E01501D11016E02501E11026E0C
:106A100003501F11036E0050182701501923025014
:106A20001A2303501B230001B35101011827000151
:106A3000B451010119230001B55101011A230001CC
:106A4000B65101011B230001D751040DF350036A15
:106A5000D80FE96E000E0320EA6EEFCF00F0ECCF06
:106A600001F0ECCF02F0ECCF03F000500101182749
:106A70000150192302501A2303501B23990E182585
:106A80000001D26F790E010119210001D36F820E2E
:106A900001011A210001D46F5A0E01011B210001CE
:106AA000D56FD651130802E3000E01D0010E01018B
:106AB000186F0001D651270802E2000E01D0010E26
:106AC00001011815D8B481D0A6C021F1A5C020F1CC
:106AD000A4C01FF1A3C01EF1050E226F0001D1DD7D
:106AE00003C01BF102C01AF101C019F100C018F176
:106AF000A751AB1901011C6F0001A851AC1901018C
:106B00001D6F0001A951AD1901011E6F0001AA51AD
:106B1000AE1901011F6F1C510001AF19006E010178
:106B20001D510001B019016E01011E510001B11982
:106B3000026E01011F510001B219036E00500101E4
:106B400018270150192302501A2303501B23000158
:106B5000B351010118270001B451010119230001AB
:106B6000B55101011A230001B65101011B23000197
:106B7000D751040DF350036AD80FE96E000E0320BD
:106B8000EA6EEFCF00F0ECCF01F0ECCF02F0ECCFEB
:106B900003F00050010118270150192302501A2355
:106BA00003501B23A10E18250001D26FEB0E01012B
:106BB00019210001D36FD90E01011A210001D46FF0
:106BC0006E0E01011B210001D56F0001D65127086F
:106BD00002E3000E01D0010E0101186F0001D65131
:106BE0003B0802E2000E01D0010E01011815D8B4D5
:106BF0009DD0A6C021F1A5C020F1A4C01FF1A3C063
:106C00001EF1050E226F00013CDD03C01BF102C026
:106C10001AF101C019F100C018F1A751AB1501011B
:106C20001C6F0001A851AC1501011D6F0001A95195
:106C3000AD1501011E6F0001AA51AE1501011F6FB4
:106C40000001A751AF15006EA851B015016EA951F2
:106C5000B115026EAA51B215036E005001011C134A
:106C600001501D1302501E1303501F130001AB519E
:106C7000AF15006EAC51B015016EAD51B115026E7D
:106C8000AE51B215036E005001011C11006E01508F
:106C90001D11016E02501E11026E03501F11036E72
:106CA000005018270150192302501A2303501B23A8
:106CB0000001B351010118270001B451010119234A
:106CC0000001B55101011A230001B65101011B2336
:106CD0000001D751040DF350036AD80FE96E000E7E
:106CE0000320EA6EEFCF00F0ECCF01F0ECCF02F022
:106CF000ECCF03F000500101182701501923025076
:106D00001A2303501B23DC0E18250001D26FBC0E82
:106D1000010119210001D36F1B0E01011A2100018D
:106D2000D46F8F0E01011B210001D56F0001D651D8
:106D30003B0802E3000E01D0010E0101186F0001B3
:106D4000D6514F0802E2000E01D0010E01011815C4
:106D5000D8B482D0A6C021F1A5C020F1A4C01FF1F3
:106D6000A3C01EF1050E226F00018BDC03C01BF1D6
:106D700002C01AF101C019F100C018F1A751AB19F6
:106D800001011C6F0001A851AC1901011D6F000128
:106D9000A951AD1901011E6F0001AA51AE190101DF
:106DA0001F6F1C510001AF19006E01011D51000140
:106DB000B019016E01011E510001B119026E0101ED
:106DC0001F510001B219036E005001011827015034
:106DD000192302501A2303501B230001B351010150
:106DE00018270001B451010119230001B551010117
:106DF0001A230001B65101011B230001D751040DD4
:106E0000F350036AD80FE96E000E0320EA6EEFCF4D
:106E100000F0ECCF01F0ECCF02F0ECCF03F000502B
:106E2000010118270150192302501A2303501B2374
:106E3000D60E18250001D26FC10E010119210001E3
:106E4000D36F620E01011A210001D46FCA0E010135
:106E50001B210001D56F0101B2C0B6F0B1C0B5F081
:106E6000B0C0B4F0AFC0B3F0AEC0B2F0ADC0B1F0DE
:106E7000ACC0B0F0ABC0AFF0AAC021F1A9C020F106
:106E8000A8C01FF1A7C01EF1020E226F00012AEC5C
:106E900033F003C0AEF002C0ADF001C0ACF000C0F2
:106EA000ABF0A6C0AAF0A5C0A9F0A4C0A8F0A3C0EA
:106EB000A7F0D5C0A6F0D4C0A5F0D3C0A4F0D2C02E
:106EC000A3F0D62BB0D451EF38F002EC19F0F2CF8A
:106ED000D0F0F29EAA6A200EA96EA69CA69EA6805D
:106EE000A850D0BFF28ED16FF2CFD2F0F29EAA6A34
:106EF000210EA96EA69CA69EA680A850D2BFF28E97
:106F0000D36FD1C0D5F0D3C0D4F0F2CFD6F0F29E7B
:106F1000AA6A220EA96EA69CA69EA680A850D6BFDD
:106F2000F28ED76FA20EF66E2E0EF76E196AF2BEB3
:106F3000198EF29E150E0101266F000130EC1AF039
:106F400019BEF28E100EE96ED5C0D9F0D4C0D8F0BB
:106F500095EC26F0BA0EF66E2E0EF76E196AF2BE9A
:106F6000198EF29E0D0E0101266F000130EC1AF011
:106F700019BEF28E196AF2BE198EF29ED7C029F19F
:106F80001B0E01012A6F00012DEC19F019BEF28EC3
:106F90000D0E04009EA8FDD7AD6E0A0E04009EA83B
:106FA000FDD7AD6E0A0E04009EA8FDD7AD6ECE0EC5
:106FB000F66E2E0EF76E196AF2BE198EF29E9EECD8
:106FC00019F019BEF28E1C0EF66E2F0EF76E196AAE
:106FD000F2BE198EF29E9EEC19F019BEF28EF2CF1F
:106FE000D0F0F29EAA6A100EA96EA69CA69EA6805C
:106FF000A850D0BFF28ED16FF2CFD2F0F29EAA6A23
:10700000110EA96EA69CA69EA680A850D2BFF28E95
:10701000D36FD1C0BBF0D3C0BAF06A0EF66E2F0E9C
:10702000F76E196AF2BE198EF29E130E0101266FD9
:10703000000130EC1AF019BEF28E100EE96EBBC0E2
:10704000D9F0BAC0D8F095EC26F00D0E04009EA839
:10705000FDD7AD6E0A0E04009EA8FDD7AD6E0A0ED8
:1070600004009EA8FDD7AD6E840EF66E2F0EF76E4F
:10707000196AF2BE198EF29E9EEC19F019BEF28EBC
:1070800017EC33F002C0B9F001C0B8F0B85303E117
:10709000B95301E189D1B9C0D1F0B8C0D0F058EFEF
:1070A00033F0BC0EF66E2F0EF76E196AF2BE198E13
:1070B000F29E9EEC19F019BEF28E1A0EF66E2A0E92
:1070C000F76E196AF2BE198EF29E9EEC19F019BE87
:1070D000F28EEA0EF66E2F0EF76E196AF2BE198E58
:1070E000F29E9EEC19F019BEF28E32EC30F001C027
:1070F000D0F032EC30F001C0D1F032EC30F001C011
:10710000D2F032EC30F0D0C0BFF0D1C0BEF0D2C06F
:10711000BDF001C0BCF032EC30F001C0D0F032EC78
:1071200030F001C0D1F032EC30F001C0D2F032ECDE
:1071300030F0D0C0C3F0D1C0C2F0D2C0C1F001C0A5
:10714000C0F032EC30F001C0D0F032EC30F001C0D1
:10715000D1F032EC30F001C0D2F032EC30F0D0C0DF
:10716000C7F0D1C0C6F0D2C0C5F001C0C4F032EC47
:1071700030F001C0D0F032EC30F001C0D1F032EC90
:1071800030F001C0D2F032EC30F0D0C0CBF0D1C042
:10719000CAF0D2C0C9F001C0C8F032EC30F001C072
:1071A000D0F032EC30F001C0D1F032EC30F001C060
:1071B000D2F032EC30F0D0C0CFF0D1C0CEF0D2C09F
:1071C000CDF001C0CCF0A351BC5DD8A4D9D0A4515E
:1071D000BD5DD8A4D5D0A551BE5DD8A4D1D0A6514F
:1071E000BF5DD8A4CDD0A751C05DD8A4C9D0A85147
:1071F000C15DD8A4C5D0A951C25DD8A4C1D0AA513F
:10720000C35DD8A4BDD0AB51C45DD8A4B9D0AC5136
:10721000C55DD8A4B5D0AD51C65DD8A4B1D0AE512E
:10722000C75DD8A4ADD0AF51C85DD8A4A9D0B05126
:10723000C95DD8A4A5D0B151CA5DD8A4A1D0B2511E
:10724000CB5DD8A49DD0B351CC5DD8A499D0B45116
:10725000CD5DD8A495D0B551CE5DD8A491D0B6510E
:10726000CF5DD8A48DD0BA51B827BB51B923B9C0CE
:10727000D0F0D16BAA6A100EA96ED0C0A8FFA69C50
:10728000A69EA684F250006EF29E0F01550EA76EC8
:10729000AA0EA76EA682A6B2FED7A6940050F2123E
:1072A000AA6A110EA96EB8C0A8FFA69CA69EA684C5
:1072B000F2CF00F0F29E550EA76EAA0EA76EA68220
:1072C000A6B2FED7A6940050F212F2CFD0F0F29EF2
:1072D000AA6A220EA96EA69CA69EA680A8500001AE
:1072E000D0BFF28E010FD16FAA6A220EA96ED1C053
:1072F000A8FFA69CA69EA684F250006EF29E0F01E7
:10730000550EA76EAA0EA76EA682A6B2FED7A694A9
:107310000050F212F00EF66E2F0EF76E196AF2BEE2
:10732000198EF29E2B0E0101266F000130EC1AF02F
:1073300019BEF28E100EE96EBBC0D9F0BAC0D8F0FB
:1073400095EC26F01E0EF66E300EF76E196AF2BE40
:10735000198EF29E040E0101266F000130EC1AF026
:1073600019BEF28E100EE96EB9C0D9F0B8C0D8F0CF
:1073700095EC26F02E0E04009EA8FDD7AD6E0CD025
:10738000280EF66E300EF76E196AF2BE198EF29E56
:107390009EEC19F019BEF28E080ED06FFA0ED16F66
:1073A00006EC20F0D02FFAD755EF41F0F3EC20F0A7
:1073B000810EC26F3BEC21F001C0B8F09CEC20F0D4
:1073C000F3EC20F0820EC26F3BEC21F001C0B9F06B
:1073D0009CEC20F08E0EF66E3D0EF76E196AF2BE32
:1073E000198EF29E150E0101266F000130EC1AF085
:1073F00019BEF28E196AF2BE198EF29EB8C026F13D
:10740000370E0101276F000146EC1AF019BEF28E0B
:107410002E0E04009EA8FDD7AD6E196AF2BE198E1D
:10742000F29EB9C026F1370E0101276F000146EC2C
:107430001AF019BEF28E3A0E04009EA8FDD7AD6E6A
:107440000A0E04009EA8FDD7AD6E0D0E04009EA886
:10745000FDD7AD6E6DEF41F0006A016ACB51D89057
:10746000CCB1002600320132CCB30026003201320A
:10747000CCB5002600320132CCB7002600320132F2
:10748000CCB9002600320132CCBB002600320132DA
:10749000CCBD002600320132CCBF002600320132C2
:1074A000BEEF3AF0C96BC76B0A0EC86FC66BC4510A
:1074B000C51103E1000E016EC1D0C951C92B036A89
:1074C000C425E96EC5510320EA6EEFCFCAF0CA5158
:1074D0002D080DE1010EC76FC951C92B036AC425E0
:1074E000E96EC5510320EA6EEFCFCAF00DD0CA5144
:1074F0002B080AE1C951C92B036AC425E96EC5519D
:107500000320EA6EEFCFCAF0CA512F08D8B08ED050
:10751000CA513908D8A08AD0CA51300821E1036A7B
:10752000C951C425E96EC5510320EA6EEF507808B1
:107530000AE0036AC951C425E96EC5510320EA6E09
:10754000EF5058080DE1100EC86FC92BC951C92B57
:10755000036AC425E96EC5510320EA6EEFCFCAF075
:10756000C8510A081BE1CA512F0817E2CA5139084D
:1075700014E30A0ECB6FC6C0CCF06ED7300ECA5DD6
:107580000124C66FC951C92B036AC425E96EC551D0
:107590000320EA6EEFCFCAF0E6D748D0C8511008F2
:1075A00045E1CA51600806E2CA517A0803E3CA51AC
:1075B000DF0B01D0CA51CA6FCA512F0803E2CA516A
:1075C000390806E2CA51400831E2CA5146082EE3A2
:1075D000CA512F080CE2CA51390809E3C639CB6FEA
:1075E000F00ECB17300ECA5DCB25C66F09D0C63959
:1075F000CB6FF00ECB17410ECA5D0A0FCB25C66FBD
:10760000C951C92B036AC425E96EC5510320EA6E2E
:10761000EFCFCAF0CA51600806E2CA517A0803E304
:10762000CA51DF0B01D0CA51CA6FC6D7C72D04D0CB
:10763000C8510A0801E1C66DC6C001F02BEF3BF04E
:10764000DA6BBE0ED96F050EDB6FC4EC31F0C56B83
:10765000BE0EC46F27D701C0C3F0C3C001F0000C39
:10766000B96BB86B02EC19F0CC0EF66E3E0EF76EED
:10767000196AF2BE198EF29E9EEC19F019BEF28EB6
:1076800017EC33F002C0BBF001C0BAF0BB510708E1
:1076900004E30BE1BA51D60808E2BB51060806E242
:1076A000FF0A03E1BA51E10801E2DED7F00EF66EFF
:1076B0003E0EF76E196AF2BE198EF29E9EEC19F01C
:1076C00019BEF28EBDDF01C0BCF0BC5303E0BC515B
:1076D0000C0801E2EBD7140EF66E3F0EF76E196A36
:1076E000F2BE198EF29E9EEC19F019BEF28EA8DF42
:1076F00001C0BDF0BD5303E0BD511F0801E2EBD74F
:10770000B9C0BEF0BF6BAA6A130EA96EBEC0A8FFB7
:10771000A69CA69EA684F250006EF29E0F01550E06
:10772000A76EAA0EA76EA682A6B2FED7A694005098
:10773000F212AA6A140EA96EB8C0A8FFA69CA69E53
:10774000A684F2CF00F0F29E550EA76EAA0EA76E89
:10775000A682A6B2FED7A6940050F212360EF66E9E
:107760003F0EF76E196AF2BE198EF29E00019EEC72
:1077700019F019BEF28EB9C0BEF0BF6B540EF66E92
:107780003F0EF76E196AF2BE198EF29E3B0E010192
:10779000266F000130EC1AF019BEF28E196AF2BEA3
:1077A000198EF29EBEC026F1370E0101276F00012F
:1077B00046EC1AF019BEF28E196AF2BE198EF29ECC
:1077C000B8C026F1370E0101276F000146EC1AF010
:1077D00019BEF28E0D0E04009EA8FDD7AD6E0A0EE6
:1077E00004009EA8FDD7AD6E84EF41F0BC6BBC5188
:1077F0007F08D8A0B9D09488050E006E002EFED761
:107800009486060E006E002EFED78B989498050E77
:10781000006E002EFED78B969496196AF2BE198ED2
:10782000F29E1AC027F193EC18F019BEF28E196A75
:10783000F2BE198EF29EBCC027F193EC18F019BE6F
:10784000F28E010E006E08EC21F001C0B8F0010EBE
:10785000006E08EC21F001C0B9F0010E006E08ECDA
:1078600021F001C0BAF0006A08EC21F001C0BBF0C1
:1078700094980000948682A6FED7050E006E002E16
:10788000FED700D000009488050E006E002EFED7B3
:10789000800EBC25BD6FAA6ABDC0A9FFB8C0A8FFF5
:1078A000A69CA69EA684F250006EF29E0F01550E75
:1078B000A76EAA0EA76EA682A6B2FED7A694005007
:1078C000F212810E0001BC25BD6FAA6ABDC0A9FFDE
:1078D000B9C0A8FFA69CA69EA684F250006EF29E98
:1078E0000F01550EA76EAA0EA76EA682A6B2FED7EE
:1078F000A6940050F212820E0001BC25BD6FAA6A48
:10790000BDC0A9FFBAC0A8FFA69CA69EA684F2503F
:10791000006EF29E0F01550EA76EAA0EA76EA682EC
:10792000A6B2FED7A6940050F212830E0001BC2529
:10793000BD6FAA6ABDC0A9FFBBC0A8FFA69CA69E3A
:10794000A684F250006EF29E0F01550EA76EAA0E8D
:10795000A76EA682A6B2FED7A6940050F212030E1E
:107960000001BC27BC2B43D702EC19F0980EF66E31
:107970003F0EF76E196AF2BE198EF29E9EEC19F058
:1079800019BEF28E040EBD6FFA0ED16F06EC20F018
:10799000BD2FFAD79CEF41F0B86BB8517F08D8A043
:1079A000B5D0F3EC20F0800EB825BB6FF2CFBCF061
:1079B000F29EAA6ABBC0A9FFA69CA69EA680A8505C
:1079C000BCBFF28EBB6FB8C0C3F0BBC0C4F058ECF4
:1079D00020F09CEC20F0B8C0C2F03BEC21F001C0DC
:1079E000B9F0800EB825BB6FF2CFBCF0F29EAA6A48
:1079F000BBC0A9FFA69CA69EA680A850BCBFF28EC5
:107A0000B95DD8B481D002EC19F0BC0EF66E3F0E11
:107A1000F76E196AF2BE198EF29E9EEC19F019BE2D
:107A2000F28E800EB825BB6FF2CFBCF0F29EAA6A30
:107A3000BBC0A9FFA69CA69EA680A850BCBFF28E84
:107A4000BB6FDE0EF66E3F0EF76E196AF2BE198E30
:107A5000F29E050E0101266F000130EC1AF019BEEE
:107A6000F28E196AF2BE198EF29EB8C026F1370E58
:107A70000101276F000146EC1AF019BEF28EE60EE6
:107A8000F66E3F0EF76E196AF2BE198EF29E080E60
:107A90000101266F000130EC1AF019BEF28E196A4E
:107AA000F2BE198EF29EB9C026F1370E0101276F82
:107AB000000146EC1AF019BEF28EF10EF66E3F0E82
:107AC000F76E196AF2BE198EF29E100E0101266F32
:107AD000000130EC1AF019BEF28E196AF2BE198E4E
:107AE000F29EBBC026F1370E0101276F000146EC64
:107AF0001AF019BEF28E080EBB6FFA0ED16F06ECAB
:107B000020F0BB2FFAD77CD1B82B47D7F2CFBBF0F0
:107B1000F29EAA6A800EA96EA69CA69EA680A85078
:107B2000BBBFF28EBA6FBA51F00FD8B061D1100F4F
:107B300002EF3FF0F3EC20F0830EC36F020EC46F30
:107B400058EC20F0B10E1A6E9CEC20F0015205E0CA
:107B5000BB6BBC6B6CEC27F002D088EC27F048D1F3
:107B6000F3EC20F0830EC36F050EC46F58EC20F0C9
:107B7000B30E1A6E9CEC20F0015205E0BB6BBC6B9F
:107B80006CEC27F002D088EC27F032D1F3EC20F037
:107B9000830EC36F010EC46F58EC20F0B50E1A6E41
:107BA0009CEC20F0015205E0BB6BBC6B6CEC27F049
:107BB00002D088EC27F01CD1F3EC20F0830EC36FC9
:107BC000060EC46F58EC20F0B70E1A6E9CEC20F035
:107BD000015205E0BB6BBC6B6CEC27F002D088EC6B
:107BE00027F006D1F3EC20F0830EC36F030EC46FB1
:107BF00058EC20F0B90E1A6E9CEC20F0015205E012
:107C0000BB6BBC6B6CEC27F002D088EC27F0F0D09B
:107C1000F3EC20F0830EC36F070EC46F58EC20F016
:107C2000BB0E1A6E9CEC20F0015205E0BB6BBC6BE6
:107C30006CEC27F002D088EC27F0DAD0F3EC20F0DF
:107C4000830EC36FC46B58EC20F0BD0E1A6E9CEC13
:107C500020F0015205E0BB6BBC6B6CEC27F002D04E
:107C600088EC27F0C5D0F3EC20F0830EC36F040E30
:107C7000C46F58EC20F0BF0E1A6E9CEC20F001523D
:107C800005E0BB6BBC6B6CEC27F002D088EC27F0F6
:107C9000AFD0F3EC20F0830EC36F020EC46F58EC2C
:107CA00020F0B10E1A6E9CEC20F0015205E0BB6B87
:107CB000BC6B6CEC27F002D088EC27F099D0F3EC89
:107CC00020F0830EC36F050EC46F58EC20F0B30E86
:107CD0001A6E9CEC20F0015205E0BB6BBC6B6CECA7
:107CE00027F002D088EC27F083D0F3EC20F0830E4D
:107CF000C36F010EC46F58EC20F0B50E1A6E9CECE9
:107D000020F0015205E0BB6BBC6B6CEC27F002D09D
:107D100088EC27F06DD0F3EC20F0830EC36F060ED5
:107D2000C46F58EC20F0B70E1A6E9CEC20F0015294
:107D300005E0BB6BBC6B6CEC27F002D088EC27F045
:107D400057D0F3EC20F0830EC36F030EC46F58ECD2
:107D500020F0B90E1A6E9CEC20F0015205E0BB6BCE
:107D6000BC6B6CEC27F002D088EC27F041D0F3EC30
:107D700020F0830EC36F070EC46F58EC20F0BB0ECB
:107D80001A6E9CEC20F0015205E0BB6BBC6B6CECF6
:107D900027F002D088EC27F02BD0F3EC20F0830EF4
:107DA000C36FC46B58EC20F0BD0E1A6E9CEC20F033
:107DB000015205E0BB6BBC6B6CEC27F002D088EC89
:107DC00027F016D0F3EC20F0830EC36F040EC46FBF
:107DD00058EC20F0BF0E1A6E9CEC20F0015205E02A
:107DE000BB6BBC6B6CEC27F002D088EC27F000D0AA
:107DF000080EBB6FFA0ED16F06EC20F0BB2FFAD73E
:107E0000B7EF41F0E824F76AF7361F0FF66E7E0EE3
:107E1000F7220A00F550FA6E0800F550F96E347B2F
:107E2000607B8C7BB87BE47B107C3C7C667C927CAA
:107E3000BE7CEA7C167D427D6E7D9A7DC47DB96BE9
:107E4000B9517F081BE3B9C0C2F03BEC21F001C07F
:107E5000B8F0196AF2BE198EF29EB8C026F1370E3C
:107E60000101276F000146EC1AF019BEF28E200EB8
:107E700004009EA8FDD7AD6EB92BE2D70D0E04000D
:107E80009EA8FDD7AD6E0A0E04009EA8FDD7AD6E6C
:107E9000E7EF41F0F86AD09E078EEA6AE96AB88691
:107EA0002A0EAF6E000EB06EA60EAC6E900EAB6ECC
:107EB0001A6A1B6A9C919C93C150C00B0F09C16E3A
:107EC000070EB46E9D6B9E6BD190C150C00B0F0915
:107ED000C16EC290C69A949A94889496010EC66E0A
:107EE000000EC76ED190810ED56ECD6A000ECA6E9F
:107EF000000ECB6E070EB46E9250926E0400100E00
:107F0000006E002EFED7B450A19CB56A03EC20F0A1
:107F1000C80ED16F06EC20F002EC00F01DEF20F04F
:107F200021EF20F02DEF20F0196AF2BE198EF29E9B
:107F300080EC1DF019BEF28ED76AD66AF294F28AEE
:107F4000C00EF212D18004009EAAFDD7AECFB7F0CA
:107F5000B751600806E2B7517A0803E3B751DF0B67
:107F600001D0B751B76F310EB75DD70FD8B03DD242
:107F7000290FF8EF41F01A5201E137D2F29A310E8F
:107F800004009EA8FDD7AD6E7C0EC36FAA0EC46F11
:107F900058EC20F0830EC36F800EC46F58EC20F0B5
:107FA000BD0E1A6E9CEC20F0015208E09C85010E7B
:107FB000BB6F800EBC6F6CEC27F002D088EC27F012
:107FC00014D21A5201E111D2F29A320E04009EA884
:107FD000FDD7AD6E7C0EC36FAA0EC46F58EC20F0B7
:107FE000830EC36F810EC46F58EC20F0B50E1A6E6D
:107FF0009CEC20F0015208E09C85010EBB6F810EC5
:10800000BC6F6CEC27F002D088EC27F0EED11A524E
:1080100001E1EBD1F29A330E04009EA8FDD7AD6EBC
:108020007C0EC36FAA0EC46F58EC20F0830EC36F92
:10803000820EC46F58EC20F0B10E1A6E9CEC20F04A
:10804000015208E09C85010EBB6F820EBC6F6CEC88
:1080500027F002D088EC27F0C8D11A5201E1C5D12F
:10806000F29A340E04009EA8FDD7AD6E7C0EC36F4D
:10807000AA0EC46F58EC20F0830EC36FC46F58EC87
:1080800020F0B90E1A6E9CEC20F0015208E09C859D
:10809000010EBB6F830EBC6F6CEC27F002D088EC36
:1080A00027F0A3D11A5201E1A0D1F29A350E0400B3
:1080B0009EA8FDD7AD6E7C0EC36FAA0EC46F58ECA0
:1080C00020F0830EC36F840EC46F58EC20F0BF0EF7
:1080D0001A6E9CEC20F0015208E09C85010EBB6FEB
:1080E000840EBC6F6CEC27F002D088EC27F07DD1B9
:1080F0001A5201E17AD1F29A360E04009EA8FDD7F9
:10810000AD6E7C0EC36FAA0EC46F58EC20F0830EC8
:10811000C36F850EC46F58EC20F0B30E1A6E9CEC42
:1081200020F0015208E09C85010EBB6F850EBC6FEC
:108130006CEC27F002D088EC27F057D11A5201E1FD
:1081400054D1F29A370E04009EA8FDD7AD6E7C0E76
:10815000C36FAA0EC46F58EC20F0830EC36F860E57
:10816000C46F58EC20F0B70E1A6E9CEC20F0015250
:1081700008E09C85010EBB6F860EBC6F6CEC27F08F
:1081800002D088EC27F031D11A5201E12ED1F29AB7
:10819000380E04009EA8FDD7AD6E7C0EC36FAA0EEC
:1081A000C46F58EC20F0830EC36F870EC46F58EC79
:1081B00020F0BB0E1A6E9CEC20F0015208E09C856A
:1081C000010EBB6F870EBC6F6CEC27F002D088EC01
:1081D00027F00BD11A5201E108D1D190F29A410E49
:1081E00004009EA8FDD7AD6EB86B010EB96F77EC99
:1081F0002DF0FCEC2FF0196AF2BE198EF29E80EC85
:108200001DF019BEF28EF294F28AD180EED01A528D
:1082100001E1EBD09CB301D0EAD0D190F29A420EAA
:1082200004009EA8FDD7AD6E04EF31F0196AF2BECE
:10823000198EF29E80EC1DF019BEF28EF294F28A35
:10824000D180D3D0F29A9C73196AF2BE198EF29E35
:1082500080EC1DF019BEF28EF294F28AC6D01A524A
:1082600001E1C3D0D190F29A460E04009EA8FDD73A
:10827000AD6E9BEF31F0FCEC2FF0196AF2BE198E57
:10828000F29E80EC1DF019BEF28EF294F28AD1803B
:10829000ACD01A5201E1A9D0D190F29A470E040055
:1082A0009EA8FDD7AD6E65EF37F0196AF2BE198E44
:1082B000F29E80EC1DF019BEF28EF294F28AD1800B
:1082C00094D01A5201E191D0D190F29A480E040054
:1082D0009EA8FDD7AD6ED6EF39F0FCEC2FF0196AF1
:1082E000F2BE198EF29E80EC1DF019BEF28EF29451
:1082F000F28AD1807AD0D190F29A490E04009EA8D9
:10830000FDD7AD6E30EF3BF0196AF2BE198EF29ECA
:1083100080EC1DF019BEF28EF294F28AD18065D005
:108320001A5201E162D0D190F29A4B0E04009EA83D
:10833000FDD7AD6EF6EF3BF0196AF2BE198EF29ED4
:1083400080EC1DF019BEF28EF294F28AD1804DD0ED
:108350001A5201E14AD09CB101D047D0D190F29A93
:108360004C0E04009EA8FDD7AD6ECCEF3CF0196A10
:10837000F2BE198EF29E80EC1DF019BEF28EF294C0
:10838000F28AD18032D0D190F29A4D0E04009EA88C
:10839000FDD7AD6E100EB86F010EB96F77EC2DF0F2
:1083A000FCEC2FF0196AF2BE198EF29E80EC1DF0E3
:1083B00019BEF28EF294F28AD18017D01A5201E1DE
:1083C00014D09CB301D013D0D190F29A38D5FCECE4
:1083D0002FF0196AF2BE198EF29E80EC1DF019BEC4
:1083E000F28EF294F28AD18000D00400ACD5030062
:1083F000E824F76AF7360B0FF66E840EF7220A00B0
:10840000F550FA6E0800F550F96E767FC27F0E8047
:108410005A80A480F0803C818881EA83EA83EA83E1
:10842000EA83EA83EA83EA83EA83D4810E82EA83D9
:10843000EA8344825E829282C282F682EA83208349
:1084400050838683EA83EA83EA83EA83EA83EA83C2
:0C845000EA83EA83EA83EA83EA83BC83C0
:020000040030CA
:0E00000000C2171E0085010007C007E0074080
:00000001FF
